:020000040800F2
:10000000D85D0020290200083D370008452E000871
:10001000DD350008710D0008114B000800000000DC
:10002000000000000000000000000000213A00086D
:100030003517000800000000B13900089945000894
:10004000430200084302000843020008430200087C
:10005000430200084302000843020008430200086C
:10006000430200084302000843020008430200085C
:100070005916000843020008430200084302000822
:10008000430200084302000843020008950D0008DF
:10009000750D0008850D00084302000843020008A2
:1000A000430200084302000843020008430200081C
:1000B000430200084302000843020008430200080C
:1000C00043020008430200084302000843020008FC
:1000D00043020008430200084302000843020008EC
:1000E00043020008430200084302000843020008DC
:1000F00043020008430200084302000843020008CC
:1001000043020008430200084302000843020008BB
:1001100043020008430200084302000843020008AB
:10012000430200084302000843020008430200089B
:10013000430200084302000843020008C50D0008FE
:10014000A50D0008B50D0008430200084302000891
:100150004302000869160008430200084302000831
:10016000430200084302000843020008430200085B
:100170004302000843020008430200080000000098
:10018000430200084302000800F002F800F03CF8C7
:100190000AA090E8000C82448344AAF10107DA45E2
:1001A00001D100F031F8AFF2090EBAE80F0013F0F8
:1001B000010F18BFFB1A43F001031847387F0000F6
:1001C000587F0000103A24BF78C878C1FAD8520787
:1001D00024BF30C830C144BF04680C6070470000C1
:1001E0000023002400250026103A28BF78C1FBD840
:1001F000520728BF30C148BF0B6070471FB507F0DA
:10020000F5FE1FBD10B510BD00F062F91146FFF7F5
:10021000F5FF04F027FD00F080F903B4FFF7F2FFCB
:1002200003BC00F083F900000948804709480047F3
:10023000FEE7FEE7FEE7FEE7FEE7FEE7FEE7FEE796
:10024000FEE7FEE704480549054A064B70470000F3
:100250005146000889010008D8570020D85D0020C9
:10026000D8590020D859002053EA020C00F06980C8
:100270002DE9F04B4FF00006002B1FBFB3FA83F5BA
:1002800003FA05F424FA05F65E4012BF1643B2FAEB
:1002900082F502FA05F4C5F120051EBF22FA05FC1D
:1002A00044EA0C04203556EA044C4FEA144418BFC3
:1002B000641C4FF000084FF00009904271EB030CF2
:1002C00039D3002919BFB1FA81F701FA07F6B0FA5C
:1002D00080F700FA07F6C7F120071EBF20FA07FCD7
:1002E00046EA0C062037B6FBF4FCA7EB0507103FE7
:1002F00007F01F0BCBF120062CFA06F60CFA0BFBCD
:1003000044BFB3460026202FA4BF5E464FF0000B2B
:100310005BEA060C08BF4FF0010B19EB0B0948EB29
:100320000608ABFB027C06FB02CC0BFB03CCC01B1C
:1003300071EB0C01C1E70B46024641464846BDE859
:10034000F08B13B5084318BF4FF0FF300146AFF3F1
:100350000080BDE81C407047032A40F2308010F056
:10036000030C00F0158011F8013BBCF1020F624450
:1003700098BF11F801CB00F8013B38BF11F8013BE1
:10038000A2F1040298BF00F801CB38BF00F8013B8E
:1003900011F0030300F02580083AC0F0088051F8FE
:1003A000043B083A51F804CBA0E80810F5E7121D09
:1003B0005CBF51F8043B40F8043BAFF30080D20728
:1003C00024BF11F8013B11F801CB48BF11F8012BF4
:1003D00024BF00F8013B00F801CB48BF00F8012B17
:1003E000704710B5203AC0F00B80B1E81850A0E873
:1003F0001850B1E81850A0E81850203ABFF4F5AFF3
:100400005FEA027C24BFB1E81850A0E8185044BF4E
:1004100018C918C0BDE810405FEA827C24BF51F8BB
:10042000043B40F8043B08BF7047D20728BF31F8AF
:10043000023B48BF11F8012B28BF20F8023B48BF00
:1004400000F8012B704702F0FF0343EA032242EA5F
:10045000024200F002B84FF0000200B51346944685
:100460009646203922BFA0E80C50A0E80C50B1F10C
:100470002001BFF4F7AF090728BFA0E80C5048BF20
:100480000CC05DF804EB890028BF40F8042B08BFBE
:10049000704748BF20F8022B11F0804F18BF00F8BA
:1004A000012B704770477047704710B500F008F88F
:1004B000006810BD10B5044600F002F8046010BDDD
:1004C00000487047180100200048704718010020BC
:1004D0007546FFF7F9FFAE4605006946534620F022
:1004E0000700854618B020B5FFF7ACFEBDE82040F8
:1004F0004FF000064FF000074FF000084FF0000BE0
:10050000AC46ACE8C009ACE8C009ACE8C009ACE84E
:10051000C00921F007018D46704710B50446AFF3BE
:1005200000802046BDE81040FFF777BE0149182043
:10053000ABBEFEE72600020070470000B1EE601A75
:10054000B4EE600AF1EE10FAB4EE401AC8BFB0EE95
:10055000600AF1EE10FAC8BFB0EE410A7047000021
:100560002DE9F04381B040F6A418C2F20008064617
:10057000D8F8000014460D466421002A08BF0A245A
:1005800004F002FD08B1FB242FE040F6A019C2F2EE
:100590000009D9F8000000E0006930B10178B142EB
:1005A000FAD14168A942F7D11AE0142000F08AFB81
:1005B00088B1074620461C21002204F04DFCB8609B
:1005C00058B1D9F800003C7300243E707D6038615A
:1005D000C9F8007005E0FE2403E0384600F06EFB29
:1005E000FF24D8F8000004F045FD60B201B0BDE87A
:1005F000F08300007047000040F6A012C2F2000233
:10060000126800E01269002A04BF002070471378C6
:100610008342F7D153688B42F4D190687047000051
:10062000D0E90212081FB0FA80F14FF0020008BFB3
:100630000320022A18BF48097047000040F2B42284
:1006400040F28C21C2F200020128C2F2000118BF60
:100650000022002818BF1146012888BF0021084643
:10066000704700002DE9F041154640F23042C2F2D9
:1006700000021278012A11D1A5B140F6A418C2F2E5
:1006800000080746D8F800000E4664211C4604F016
:100690007BFC58B1FB2040B2BDE8F081FD2040B2A8
:1006A000BDE8F081FE2040B2BDE8F0813846314619
:1006B000FFF7A2FFD8F800100646084604F0DAFC5F
:1006C00066B1304629460022234604F081FB00280B
:1006D00018BF4FF0FF3040B2BDE8F081FC2040B2BF
:1006E000BDE8F0812DE9F0478AB040F23047C2F210
:1006F0000007387808B1FD248AE040F27810C2F291
:1007000000006821FFF7A7FE002400BFE0B200F060
:100710003BFA0134012CF9D040F22C4040F2F55163
:10072000C2F20000C0F6000101600020002404F0C5
:1007300055FC40F6A411C2F200010028086066D002
:10074000E8464FF001094046282187F80090FFF75E
:1007500082FE40F28C26C2F200064FF00E0A3046AE
:100760004146CDE90244CDE90799CDF824A004948F
:1007700001F044F8304601F00FFC40F69102C0F65B
:1007800000020020062100F051F840F62535C0F6A1
:100790000005002000212A4600F048F80020012131
:1007A0002A4600F043F8002002212A4600F03EF8D5
:1007B0003046032100F0C4FF40F2B426C2F2000626
:1007C00030464146CDE9049A01F018F8304601F070
:1007D000E3FB40F65512C0F600020120082100F0AC
:1007E00025F8012000212A4600F020F801200121EF
:1007F0002A4600F01BF8012002212A4600F016F8D4
:100800003046112100F09CFF87F8009000E0FF24A3
:1008100060B20AB0BDE8F08780B540F22C42C2F267
:1008200000021268002A18BF904780BD40F2304392
:10083000C2F200031B78012B1EBFFD2358B2704784
:100840003AB101284FF0FF0398BF0C2904D958B2E0
:100850007047FE2358B2704740F2781CC2F2000C79
:10086000342310FB03C0002340F8212058B2704706
:1008700080B540F23043C2F200031B78012B03D154
:10088000FFF76EFE40B280BDFD2040B280BD00008B
:100890002DE9F04F93B003A80D3001904FF0000AFE
:1008A0000CAE002005E000BF0298002800F1010016
:1008B0004CD15FFA80FB02905846FFF7BFFE00283C
:1008C000F2D0044609E000BF01F040FE099038462E
:1008D00003A90022002304F00FFB2046002101F0B1
:1008E0000FF80028E0D02046002132460AAB01F084
:1008F00017F80028F1D10E980028304618BF0430B0
:1009000005683046FFF78CFE804628464146FFF7D3
:1009100083FF814658464946FFF76EFE0028DCD02B
:100920000746DDE90F02CDF80CA00028CDE908AAA2
:10093000CDE906AA8DF80C80CDE904598DF8182070
:10094000C2D101980AA9FFF707FDBDE713B0BDE8C2
:10095000F08F00002DE9F04F93B003A80D30019007
:100960004FF0000A0CAE002005E000BF02980028FE
:1009700000F101004CD15FFA80FB02905846FFF76E
:100980005DFE0028F2D0044609E000BF01F0DEFD64
:100990000990384603A90022002304F0ADFA20464E
:1009A000012100F0ADFF0028E0D0204601213246B1
:1009B0000AAB00F0B5FF0028F1D10E9800283046B0
:1009C00018BF043005683046FFF72AFE80462846E7
:1009D0004146FFF721FF814658464946FFF70CFE86
:1009E0000028DCD00746DDE90F02CDF80CA0002876
:1009F000CDE908AACDE906AA8DF80C80CDE9045905
:100A00008DF81820C2D101980AA9FFF7A5FCBDE70F
:100A100013B0BDE8F08F00002DE9F04389B0174610
:100A200040F23042C2F200021278012A04D1044698
:100A3000012806D9FF2000E0FD2040B209B0BDE842
:100A4000F08301F0FE001D460E46022802D00DB9CB
:100A5000FE20F2E7DDF84080B8F1080F01D9FF2051
:100A6000EBE72046FFF7EAFD98B181460020032E10
:100A70000890CDE90600CDE90400CDE9020001901F
:100A800009D8DFE806F0020A0D11019700210020C5
:100A90000DE0FE20D1E7FF20CFE70297002005E020
:100AA00001970220002102E0022002970421CDE9F3
:100AB00003100020002DCDF814808DF8180018BF09
:100AC000B8F1000F05D001A8183029464246FFF7BB
:100AD00043FC484600F0B6FF38B101A901F1180205
:100AE0006B46484600F040FE28B101A9204600F0C0
:100AF000A5F80138A1E700209FE7000079B180B593
:100B000082B00A6891F804C04B1D0021CDF800C0E6
:100B1000FFF782FF02B0BDE8804040B27047FE2080
:100B200040B270472DE9F04389B001AC04F11809D7
:100B30000025E84604E000BF002D05F1010520D1A5
:100B4000EFB23846FFF77AFD0028F5D0064600BF21
:100B5000384600F027F80028EED1304600F072FF4A
:100B60000028E9D03846214600F02EF80028E3D0CE
:100B7000304621464A46434600F0F6FD0028E7D0BD
:100B8000DAE709B0BDE8F08340F6E43100EBC010CD
:100B9000C2F2000101EBC0000021C0F80014C0F84F
:100BA0000414704740F6E43100EBC010C2F20001BB
:100BB00001EBC000D0F80014D0F80404081AB0FA11
:100BC00080F0400970470000002904BF00207047F2
:100BD0002DE9F04140F6E43C00EBC012C2F2000CFB
:100BE0000CEBC202D2F800E4D2F804349E451FD0C8
:100BF00002F204452C6800EBC0100CEBC00000EBC7
:100C00004412640150F804C0D2E901805769D2E966
:100C10000364C1E900C8C1E90447C1E90206D2E999
:100C20000620C1E906202868013000F01F00286076
:100C3000BEEB030018BF0120BDE8F08101284FF092
:100C4000000238D8B9B32DE9F04740F6E43C00EB98
:100C5000C012C2F2000C0CEBC202D2F80034D2F87F
:100C600004E4013303F01F0373451ED002F58069CD
:100C7000D9F8004000EBC0100CEBC00000EB4412B0
:100C80004FEA441AD1E904C6D1E90078D1E9025407
:100C900040F80A705661C2E9034CC2E90185D1E906
:100CA0000610C2E90610C9F80030B3EB0E0218BFF7
:100CB0000122BDE8F04710467047000080B505F0FE
:100CC00057F980BD80B504F0DDFF80BD2DE9F0410E
:100CD00004F014F8044606F005FB4FF47A784EF25F
:100CE0001806B8FBF4F4CEF20006376804FB00F5F2
:100CF00006F0F8FA60433168854208BF394656F875
:100D0000042C01FB08F10132B1FBF2F100FB08F009
:100D1000401A00F57A700021BDE8F08140F2E4321B
:100D200040F29C31C2F200020128C2F2000118BF59
:100D30000022002818BF1146084670473AB1012822
:100D40004FF0FF0398BF082904D958B27047FE231B
:100D500058B2704740F2EC1300EBC000C2F200033F
:100D600003EB8000002340F8212058B270470000B8
:100D7000FEE7000080B540F28C20C2F2000000F0D7
:100D800075FE80BD80B540F28C20C2F2000000F0FC
:100D90006DFE80BD80B540F28C20C2F2000000F0F4
:100DA00065FE80BD80B540F2B420C2F2000000F0C4
:100DB0005DFE80BD80B540F2B420C2F2000000F0BC
:100DC00055FE80BD80B540F2B420C2F2000000F0B4
:100DD0004DFE80BD4FF0030160B146F20042006855
:100DE000C4F2000202F58063984208BF0121801A14
:100DF00008BF0146C8B2704700284FF0FF0218BF75
:100E0000002901D150B2704780B590ED010A9FEDE5
:100E1000793A90ED021A30EE030A9FED773A9FED92
:100E2000775A30EE000A90ED032A80EE036A31EE25
:100E3000050A9FED731A9FED735A30EE000A90ED8C
:100E4000044A80EE011A32EE050A9FED6F2A9FEDEB
:100E50006F5A30EE000A80EE022A34EE050A30EEB8
:100E6000000A80EE035ABFEE000A36EE006A81EDFA
:100E7000016A31EE004A81ED024AB0EEC44A32EE18
:100E8000003A9FED632A81ED033A35EE001AB0EE89
:100E9000C65AB4EE425AF1EE10FAB4EE424AB0EE3F
:100EA000C33A81ED041ADCBF00224A60F1EE10FA69
:100EB000B4EE423AB0EEC11ADCBF00228A60F1EE15
:100EC00010FAB4EE421ADCBF0022CA60F1EE10FA4A
:100ED000DCBF00220A6191ED012AB7EE001AB0EEE4
:100EE000C23AB4EE413AF1EE10FA0ADBB5EE402A0E
:100EF000B0EE402AF1EE10FAC8BFB0EE412A81ED03
:100F0000012A91ED022AB0EEC23AB4EE413AF1EE76
:100F100010FA0ADBB5EE402AB0EE402AF1EE10FAE4
:100F2000C8BFB0EE412A81ED022A91ED032AB0EE4E
:100F3000C23AB4EE413AF1EE10FA0ADBB5EE402ABD
:100F4000B0EE402AF1EE10FAC8BFB0EE412A81EDB2
:100F5000032A91ED042AB0EEC23AB4EE413AF1EE22
:100F600010FA08DBB5EE402AF1EE10FAC8BFB0EE79
:100F7000410A81ED040AD1E9032301F11407D1E903
:100F800001CE87E80C5090F800E0BEF1000F02D0CF
:100F9000C37E012B20D100234B70807D831EB3FACA
:100FA00083F35A09431EDBB2022B8A700AD8DA0097
:100FB0004FF0011323FA02F2012881F8242001D115
:100FC000012000E00020002281F8250081F800E0E7
:100FD000BDE8804050B27047037E013BDBB2022B7C
:100FE000DBD84FEAC30C40F20313C0F2020323FA2A
:100FF0000CF3D1E7000051C30060AD44000032C3E0
:101000000020AC44000052C30040AD4400005DC36A
:10101000CDCC4C3D002864D02DE9F0472DED088B58
:101020008246406990F80480B8F1000F5CD008EB6C
:1010300088009FED6F8A9FED6F9A4FEA4009002765
:101040000425B7EE00AABFEE00BA002600242BE06C
:10105000DAF82000DAF84811284490ED000AC8199F
:1010600001F0F2FE80EE091ADAF87C00DAF884105A
:10107000304480ED000A0A348819043620371035D0
:10108000B4EE4A1AF1EE10FAC8BFB0EE4A1AB4EE46
:101090004B1AF1EE10FAB8BFB0EE4B1A38EE018AD7
:1010A000A14580ED001A21D0DAF81400C06A20446E
:1010B00002F02AF9DAF81400C06A204402F03EF87F
:1010C0000028C5D0DAF8201000F12C0E9EE8085058
:1010D000806B01EB860241F82630C2E901CED06078
:1010E000B6E7FF2040B270479FED418A00EE108ABC
:1010F000B8EEC00A88EE000ADAF8140030308AED43
:10110000220A02F001F9DAF81400303002F016F881
:1011100001460AF128005022FFF763F9DAF81400BB
:101120009AED1C1A90ED020A20EE010AB5EE400A73
:10113000F1EE10FA8AED1E0A0BDA9FED2F1A00BFAE
:1011400030EE010AB5EE400AF1EE10FAF8DB8AED56
:101150001E0A9AED1E0A9FED281AB4EE410AF1EE1E
:1011600010FA0ADB9FED252A30EE020AB4EE410A9E
:10117000F1EE10FAF8DA8AED1E0A9AF8500000280B
:101180001CBF31EE400A8AED1E0A9AED0D0A0AF5DF
:10119000A87001F059FE9AED0D1A9FED192A8AEDFB
:1011A000200A81EE021AB7EE000AB4EE401AF1EE00
:1011B00010FAC8BFB0EE401ABFEE000ADAF82000FD
:1011C000B4EE401AF1EE10FAB8BFB0EE401A90ED4E
:1011D000010A90ED052A8AED231A30EE420A8AEDC3
:1011E000640A0020BDEC088BBDE8F04740B27047B0
:1011F0000000000000C0DA45DB0FC940DB0FC9C0AA
:1012000000409C4590ED001AF5EE400AF1EE10FA10
:1012100031EE000A10DDB4EE600AF1EE10FAA2BF62
:1012200030EE600A80ED000A7047B5EE400AF1EE3C
:1012300010FAB8BF30EE200A80ED000A70470000B7
:10124000B5EE401AF1EE10FA30EE600AD8BF7047E2
:10125000B6EE002A21EE022AB4EE420AF1EE10FAAE
:10126000C4BF30EE410A7047B1EE422AB4EE420AE2
:10127000F1EE10FAB8BF30EE010A704740F20400F8
:10128000C2F20000704700002DE9F04381B040F247
:101290000409C2F20009D9F80450D9F8186005EB26
:1012A00085004000FFF70EFD0028C9F82C0043D050
:1012B000B000FFF707FD0028C9F81C0040D0012D41
:1012C00027DB4FF0000C40F2012E4FF01B080123EA
:1012D00000210020421ED4B2D9F82C60052C4FF01A
:1012E000000402F01F025EFA80F738BF012428FADA
:1012F00002F201EB81010130224006EB410406F8C5
:101300001130C1B28D4267802371627184F806C0CA
:10131000E0DCD9F82C10D9F81C0001220A728A747A
:101320000A7781F8262081F8302081F83A204FF0A2
:101330007E510160002006E0FFF7C0FCFF2002E0C4
:10134000FFF7BCFCFF2040B201B0BDE8F083000015
:10135000B0B5E8B140F23144C2F20004207810B1D7
:10136000FD2568B2B0BD03F043FF40F6E031C2F2A4
:101370000001086060B141F21162C0F60002002075
:1013800003210025FFF7DAFC0120207068B2B0BD10
:10139000FE2568B2B0BD00002DE9F04F82B090F894
:1013A00002C0C27840F6A8134FEADC04C2F2000380
:1013B00062F34A1490F8019005795C80C27846790E
:1013C000AD0045EA921206F0010542EA85229A80B4
:1013D000457987796E0867F3CA16DE808579C77903
:1013E0004FEA151E67F30A1EA3F808E0077A90F883
:1013F0000780457A7F0047EAD81705F0030547EADA
:10140000452BA3F80AB0457A877A4FEA950867F327
:101410008A18A3F80C80C77A857AFF0047EA551529
:10142000DD8190F80CA0477B009567F30A2AA3F8AA
:1014300010A0477B857BFF0865F34A175F82019701
:10144000C77B6CF30A2990F80EC0057CBF0047EA01
:101450009C1705F0010547EA852CA3F814C0057C0C
:10146000477C680800EE104A01EE102A02EE106A6E
:10147000AEF22D1203EE109A67F3CA10C72AB8EE27
:10148000C33AB8EEC00AB8EEC11AB8EEC22AA3F841
:101490000090D88281ED012A81ED021A81ED033A94
:1014A00081ED040A01D201220DE0AEF5FA72B2F527
:1014B0007A7F01D2032206E0AEF2DC520023C82A72
:1014C00038BF01235A00ABF22D13DDE900679BB250
:1014D000C72B0A7501D201220FE0ABF5FA7292B266
:1014E000B2F57A7F01D2032207E0ABF2DC5292B26E
:1014F0000023C82A38BF01235A00A8F22D13C72B96
:101500004A7501D201220DE0A8F5FA72B2F57A7F90
:1015100001D2032206E0A8F2DC520023C82A38BF19
:1015200001235A00A6F22D13C72B8A7501D202227D
:101530000CE0A6F5FA72B2F57A7F01D2032205E03B
:10154000A6F2DC530022C82B38BF0122AAF22D13C9
:10155000C72BCA7501D202220CE0AAF5FA72B2F5C5
:101560007A7F01D2032205E0AAF2DC530022C82BC5
:1015700038BF0122A7F22D13C72B0A7601D202220F
:101580000CE0A7F5FA72B2F57A7F01D2032205E0EA
:10159000A7F2DC530022C82B38BF0122ACF22D1376
:1015A0009BB2C72B4A7601D201220FE0ACF5FA724A
:1015B00092B2B2F57A7F01D2032207E0ACF2DC529C
:1015C00092B20023C82A38BF01235A00A0F22D137B
:1015D000C72B8A7601D202220CE0A0F5FA72B2F58E
:1015E0007A7F01D2032205E0A0F2DC530022C82B4F
:1015F00038BF0122B0F59670CA7618BF0120B9F540
:101600007A7218BF01221040087002B0BDE8F08F56
:1016100080B540F6E030C2F200000068802103F09F
:1016200049FD80BD10B504460020FFF777FB214639
:10163000192201F0C9FB002818BF4FF0FF3010BD80
:1016400080B502468020012103F074FD8038B0FA95
:1016500080F0400980BD000080B540F2DC20C2F27D
:10166000000000F045FD80BD80B540F23C30C2F284
:10167000000000F03DFD80BDD0F800C06FF00F020B
:101680004AF6AB2352FA8CF2CAF6AA230146A2FB11
:101690000330000905A31B5C40F2FF302CEA000078
:1016A0005F2A88BF0430C1E9160370470006101690
:1016B000000610168269816AB2F5005F06D06AB929
:1016C000022912D0012914D0D1B90EE0032917D86C
:1016D000DFE801F0020B020F0120704703293CBF35
:1016E000012070471CBF00207047C06AC0F3006033
:1016F0007047C06AA0F1C070B0FA80F0400970472E
:101700000020704780B5D0F800C0D0F808E0DCF8C1
:101710000000BEF1400F20F48020CCF80000084605
:10172000CCF8043004BF10460A46CCF80800CCF8C8
:101730000C2080BD7047000072B600BFFEE70000BD
:1017400090F82020013A012A04D8006800F1140220
:10175000002004E000F1240201204FF480211368EE
:10176000194311607047000010B590F820E0D0F8E0
:1017700000C0AEF1010EBEF1010FDCF808E00ED89A
:101780001EF0E05F11D0CEF3016E012000FA0EF0E2
:1017900018608B687BB1486843EAC0030DE000F134
:1017A000240101204FF4802223E000F124010120D4
:1017B0004FF400121DE008684305D1E90304034318
:1017C0000CEB0E10C0F88031C0F88441097D01296E
:1017D00005D100F5C2710B6843F480730B6051684A
:1017E000C0F88C11126800F5C071C0F88821002083
:1017F00001220B681A430A6010BD0000B0B590F8D2
:101800002020013A012A2FD846F20060C4F20000DD
:10181000026842F001020260026822F47C52026017
:10182000D1F814E0CC694A6A0368012C43EA022229
:1018300002600EF01F024FF0010303FA02F2C369C7
:101840006FEA020C23EA0203C36113D02CBBC36806
:1018500003EA0C03C360CB688C8844EA034300EBC3
:10186000CE0423640B4611E0416A41F480214162B9
:101870000120B0BDC3681343C3600B688C8844EA81
:10188000034300EBCE04236401F10C038C681B8836
:1018900043EA044300EBCE04636443688D6943EA82
:1018A0000204D1F810E0096A002D08BF03EA0C0415
:1018B00044604369BEF1000F43EA020408BF03EA33
:1018C0000C040129446102D1C1691143C16101685D
:1018D00021F0010101600020B0BD000080B5FFF7DC
:1018E00079FA032808BF80BD40F27811C2F20001E6
:1018F000342210FB0210006B002818BF804780BD07
:1019000090F82020013A012A84BF00207047006827
:101910001022002908BF0C22805800F003007047F5
:1019200010B590F82040013C012C0AD8046871B130
:101930002469A4070ED100F1240101204FF4001204
:1019400076E000F1240101204FF4802270E0E46889
:10195000A40771D0046804EB011CDCF8B0410CF55D
:10196000D87E14F004049460DCF8B04119BFE40898
:101970005460640D1460DEF800400CF5DA7E04F06B
:101980000204D460DCF8B44124075ABFDEF80040FA
:1019900004F00F0408241461DEF800400029C4F3A9
:1019A00007249461DEF800404FEA14445461DCF8E7
:1019B000B8211A70026802EB0112D2F8B8214FEA7E
:1019C00012225A70026802EB0112D2F8B8214FEAD3
:1019D00012429A70026802EB0112D2F8B8214FEA63
:1019E0001262DA70026802EB0112D2F8BC211A719D
:1019F000026802EB0112D2F8BC214FEA12225A719E
:101A0000026802EB0112D2F8BC214FEA12429A712D
:101A1000026802EB0112D2F8BC214FEA1262DA71BD
:101A2000006814BF00F1100100F10C010020202219
:101A30000B681A430A6010BD00F1240101204FF425
:101A40000012F5E790F820100139012984BF002029
:101A500070470068816882688068C1F38061C2F362
:101A6000C0621144C0F30070084470472DE9F04F84
:101A700081B0044600684669D0F804908768D0F8C1
:101A80000CB0D0F810A0D0F81880F10703D10025D1
:101A900030071CD423E0F90710D00121BA07816078
:101AA00009D4780700F1AA80380700F1B0802046F9
:101AB00000F0A0FA02E0204600F0AEFA0025F8059A
:101AC00000F18480F80300F1AA80300707D51BF0ED
:101AD000100004D0206845F400751021C160700723
:101AE00008D51BF0080005D020680821C1602046F9
:101AF00000F0F8F9B00706D52068C068800702D06A
:101B0000204600F001FA700607D51AF0100004D044
:101B1000206845F4806510210161B00608D51AF0EF
:101B2000080005D0206808210161204600F0FEF978
:101B3000F00606D520680069800702D0204600F034
:101B400007FAB00308D519F0100005D0206810215D
:101B50004160204600F00EFAF00308D519F00800A5
:101B600005D0206808214160204600F0AFFA30041B
:101B700040F18F805FEA497040F1888006F4807000
:101B800008EA102028435FEA8871014648BF41F007
:101B90000201B20558BF01465FEA48700D4648BFD2
:101BA00045F00405700558BF0D4630056ED518F098
:101BB00070006BD010380009052862D8DFE800F00B
:101BC000035356595C5F45F008055AE020684FF40E
:101BD0008071BA0581600AD4780512D4380519D409
:101BE000204600F02BFAF8037FF56FAF17E0204690
:101BF00000F036FAF8037FF568AF10E04FF40065A7
:101C00005DE705F50055F8037FF55FAF07E04FF49A
:101C1000805554E705F58045F8037FF556AF2068F9
:101C20004FF48031BA0381600AD478030FD43803AB
:101C300013D4204600F026FA30073FF548AF4EE7B0
:101C4000204600F031FA30073FF541AF47E705F590
:101C5000004530073FF53BAF41E705F580353007DC
:101C60003FF535AF3BE745F010050AE045F02005AC
:101C700007E045F0400504E045F0800501E045F44B
:101C800080752068816921F07001816120680421DC
:101C900041602DB1606A284360622046FFF71EFE56
:101CA00001B0BDE8F08F0000B0B5C8B1044690F8AF
:101CB000200010B9204600F071F82068016841F05A
:101CC0000101016000F042FC054600BF2068416848
:101CD000C90707D100F03AFC401B0B28F6D312E0ED
:101CE0000120B0BD016821F00201016000F02EFC6E
:101CF000054600BF2068416889070DD500F026FC25
:101D0000401B0B28F6D3606A052140F40030606266
:101D1000012084F82010B0BD217E0268012922F044
:101D2000800208BF80320260617E0268012922F0D1
:101D3000400208BF40320260A17E0268012922F001
:101D4000200208BF20320260E17E0268012922F0F1
:101D5000100218BF10320260217F0268012922F0B0
:101D6000080208BF08320260617F0268012922F080
:101D7000040208BF04320260D4E901C2D4E9033589
:101D800061691A432A431143ACF101021143C16155
:101D900000200121606284F82010B0BD70B586B0CB
:101DA000006846F60002C4F2000200219042CDE92C
:101DB0000411CDE90211019137D046F20041C4F27D
:101DC0000001884240F08C8040F2E011C2F2000134
:101DD0000A6843F64000C4F20200531C0B6052B97B
:101DE00000210091016841F000710160016801F07B
:101DF0000071009100990021009150F8101C1524E9
:101E000041F0080140F8101C50F8100C142500F0A7
:101E10000800009000980320019040F20040C4F2B6
:101E2000020000F50060132637E043F64000C4F2DC
:101E300002000091016841F080610160016801F0D9
:101E400080610091009940F2E011C2F200010A683D
:101E5000531C0B6052B900210091016841F00071E0
:101E60000160016801F0007100910099002100916A
:101E700050F8101C412441F0020140F8101C50F8A9
:101E8000100C402500F002000090009860200190A6
:101E900040F200403F26C4F20200022102910021DC
:101EA0000391032104910921059101A900F080FA11
:101EB00030460521002200F0C9FB304600F0C2FB8D
:101EC00028460521002200F0C1FB284600F0BAFB9D
:101ED00020460521002200F0B9FB204600F0B2FBAD
:101EE00006B070BD80B5FEF775FF032808BF80BD42
:101EF00040F27811C2F20001342210FB0210C069D6
:101F0000002818BF804780BD80B5FEF763FF032817
:101F100008BF80BD40F27811C2F20001342210FBEC
:101F200002108069002818BF804780BD80B5FEF789
:101F300051FF032808BF80BD40F27811C2F20001B2
:101F4000342210FB0210406A002818BF804780BD71
:101F500080B5FEF73FFF032808BF80BD40F278112F
:101F6000C2F20001342210FB0210006A002818BFE0
:101F7000804780BD80B5FEF72DFF032808BF80BDD8
:101F800040F27811C2F20001342210FB0210806A84
:101F9000002818BF804780BDB0B5044690F82000E7
:101FA00001281DD1022084F820002068016821F05A
:101FB0000101016000F0CAFA054600BF20684068D0
:101FC000C00713D000F0C2FA401B0B28F6D3606A9A
:101FD00040F400306062052084F820000120B0BD8C
:101FE000606A40F4002060620120B0BD00206062A1
:101FF000B0BD000080B5FEF7EDFE032808BF80BD30
:1020000040F27811C2F20001342210FB0210C068C5
:10201000002818BF804780BD80B5FEF7DBFE03288F
:1020200008BF80BD3421484340F27811C2F200015C
:102030000858002818BF804780BD000080B5FEF713
:10204000C9FE032808BF80BD40F27811C2F200012A
:10205000342210FB02100069002818BF804780BDA1
:1020600080B5FEF7B7FE032808BF80BD40F27811A7
:10207000C2F20001342210FB02104068002818BF91
:10208000804780BD80B5FEF7A5FE032808BF80BD50
:1020900040F27811C2F20001342210FB02104069B4
:1020A000002818BF804780BD80B5FEF793FE032847
:1020B00008BF80BD40F27811C2F20001342210FB4B
:1020C00002108068002818BF804780BD80B5FEF7E9
:1020D00081FE032808BF80BD40F27811C2F20001E2
:1020E000342210FB0210C06A002818BF804780BD50
:1020F000F0B581B004460020009040F20000C2F22A
:1021000000000268D4E9166048F2B5133768082168
:10211000C1F64E3381403942A2FB03250CD0226820
:1021200013685B0708D5136823F004031360B160DC
:10213000616D41F00101616501218140394208D0A2
:1021400022685269120604D5B160616D41F0020146
:10215000616504218140394208D0226812689207E3
:1021600004D5B160616D41F00401616510218140C9
:10217000394215D020680268120711D5B160026893
:102180000168520306D4C90506D4016821F008018C
:10219000016001E0080342D4216C09B12046884760
:1021A000E16D202000FA01F23A4244D02068036831
:1021B000DB0640D5B26094F835300268052B1ED19D
:1021C00022F016020260426922F080024261226C13
:1021D0000AB9A26C1AB1026822F0080202603F201C
:1021E0008840B060012084F83500216D002000296E
:1021F00084F8340040D02046884701B0F0BD016823
:10220000520310D4C90512D4016821F010010160F5
:10221000012084F83500002084F8340007E0A16C28
:102220000029BBD1BCE7080301D4616C00E0E16B7D
:1022300009B120468847606DF0B1606DC00717D0C6
:10224000052084F835002068A90A026822F00102FE
:10225000026000BF009A01328A42009202D80268EE
:10226000D207F7D1012084F83500002084F834002B
:10227000E16C09B12046884701B0F0BD2DE9F0417D
:10228000044600F063F9C4B10546022084F8350025
:102290000020216884F83400086820F001000860FC
:1022A00026683068C0070BD000F050F9401B0528A5
:1022B000F6D903212022032042E00120BDE8F0816D
:1022C000306848F23F01CFF21001251D00EA010CF1
:1022D0002ECDD4E9050E41EA0C01114319432943DF
:1022E000D4E90778084340EA0E01606A39430428BC
:1022F00041EA080103D1D4E90B23114319433160AA
:102300007169042821F0070141EA00050CD1D4E9E4
:102310000A1045EA010538B12046FFF7CBF918B19C
:102320000121402201200BE020467561FFF7A4F94E
:10233000E16D3F2202FA01F18160002201210020BB
:10234000626584F83510BDE8F0810000B0B5044640
:1023500090F83400012828D0012084F83400A56DBD
:1023600094F8350001281DD1022084F835000020A2
:1023700060652046FFF7C6F9E26D3F23206803FA47
:1023800002F2216CAA60026842F01602026019B1E2
:10239000016841F008010160016841F0010101603C
:1023A0000020B0BD002084F834000220B0BD000041
:1023B0002DE9F04F83B000F13E4202F1FF724FEA87
:1023C000B22241F600470192C4F2020708224FF000
:1023D000010E00254FF0000A4FF00008B84208BF78
:1023E000072200920AE000BF08F101080AF1040A7E
:1023F000B8F1100F05F1020500F0A4800C680EFA88
:1024000008FB14EA0B09EFD04C6804F0030CACF1A4
:10241000010EBEF1010F11D80322876802FA05F6FA
:10242000CA68B743AA403A4382604268C4F30017BF
:1024300022EA0B0207FA08F73A434260BCF1030FA5
:102440001CD0C26803238E6803FA05F7BA4306FA64
:1024500005F73A43BCF1020FC2600FD16FF00302DF
:1024600002EA580202440AF01C060F23176A03FA14
:1024700006F40B69A743B3403B431362026803238E
:102480004F68AB409A4307F00303AB401A4317F47D
:10249000403F4FF0010E0260A6D0002243F64403F5
:1024A0000292C4F202031A6843F6004442F48042E6
:1024B0001A601A68C4F2010402F480420292029A7D
:1024C00028F003024FF6084B2244CFF6FF7B52F868
:1024D0000B300AF00C070F26BE4023EA060C019BC6
:1024E000009E072B38BF1E4606FA07F747EA0C0383
:1024F00042F80B30A2684B6842EA090743F60C4CDD
:10250000DE0258BF22EA0907A760C4F2010CDCF81A
:1025100000209E0242EA090758BF22EA0907CCF8C8
:10252000007062689E0342EA090758BF22EA090761
:1025300067602268DB0342EA090358BF22EA090305
:10254000236051E703B0BDE8F08F000044F6FC7053
:10255000C2F200000068704740F20C1044F6FC71B3
:10256000C2F20000C2F2000100780A68104408605C
:102570007047000080B543F60040C4F202000168D5
:1025800041F400710160016841F4806101600168FB
:1025900041F480710160032000F068F80F2000F022
:1025A00005F800F02BF8002080BD0000B0B540F227
:1025B0000C12C2F2000240F200011278C2F20001D5
:1025C0004FF47A730968B3FBF2F20446B1FBF2F1FF
:1025D000084600F001FB0F2C4FF001050CD858B94C
:1025E0004FF0FF3021460022002500F02FF840F286
:1025F0001010C2F2000004602846B0BD80B582B061
:10260000002043F640010190C4F202014A6842F4FE
:1026100080424A604A6802F480420192019A009026
:102620000868002240F08050086008680F2100F020
:102630008050009000986FF0010000F007F802B0A1
:1026400080BD000080B502F07DFA80BD70B51446F3
:102650000D46064602F086FA2946224601F070F839
:102660000146304602F086FA70BD000080B502F0E7
:102670009BFA80BD2DE9F041002800F08B8043F6E5
:102680000808C4F202080446D8F8F8030D4600F022
:102690000700884207D288F8F853D8F8F80300F00A
:1026A0000700A84276D12068810717D5410705D5D4
:1026B000D8F8001041F4E051C8F80010010705D522
:1026C000D8F8001041F46041C8F80010D8F80010A4
:1026D000A26821F0F0011143C8F80010C0073FD1F3
:1026E000D8F8F80300F00700A84207D988F8F85393
:1026F000D8F8F80300F00700A8424BD12068410742
:1027000007D5D8F80010E26821F4E0511143C8F869
:102710000010000708D5D8F80000216920F46040B7
:1027200040EAC100C8F8000000F07EF8D8F80010B8
:1027300048F22802C1F30311C0F60002515C40F2D6
:10274000000220FA01F140F21010C2F2000000680D
:10275000C2F200021160FFF729FF0020BDE8F081FE
:102760006068811E022907D258F8081C89015CBFE5
:102770000120BDE8F08110E0012807D158F8081CBD
:1027800089035CBF0120BDE8F08106E058F8081C11
:10279000890702D40120BDE8F081D8F8001021F0AB
:1027A00003010843C8F80000FFF7D0FE064641F2D7
:1027B000883700BFD8F80000616800F00C00B0EB6B
:1027C000810F8DD0FFF7C2FE801BB842F2D90320E3
:1027D000BDE8F08140F20000C2F2000000687047DE
:1027E00080B5FFF7F7FF43F60801C4F2020109685C
:1027F00048F23802C1F38221C0F60002515CC840A1
:1028000080BD000080B5FFF7E5FF43F60801C4F284
:102810000201096848F23802C1F34231C0F60002F1
:10282000515CC84080BD000010B543F60404C4F2FA
:102830000204606800F00C0008280AD0042819BFC0
:1028400042F20040C0F2F40041F60030C0F2B7009E
:1028500010BD206821682368490241F60031C0F2AA
:10286000B70100F03F02C3F388105CBF42F20041A1
:10287000C0F2F401A1FB00010023FDF7F5FC216883
:102880000222C1F3014102EB4101B0FBF1F010BDA6
:102890002DE9F04182B0002800F0A28004460078C3
:1028A00043F60006C007C4F2020643D0B06800F049
:1028B0000C00042805D1306880033BD56068C8BB94
:1028C0008EE0B06800F00C00082802D17068400269
:1028D000F1D46568B5F5A02F0AD0B5F5803F0BD0CF
:1028E000306820F480303060306820F4802006E0CA
:1028F000306840F480203060306840F480303060D0
:10290000FFF724FE002D054611D000BF306880037C
:1029100010D4FFF71BFE401B6428F7D922E100BF4B
:10292000FFF714FE401B64284FF0030055D83068B1
:102930008003F5D4207880071AD5B06810F00C0F0A
:1029400009D0B06800F00C00082840F08A80706858
:10295000400200F186803068800702D5E0680128D7
:102960003ED13068216920F0F80040EAC1003060B3
:102970002078000738D4207840074CD4A5695DB38F
:10298000B06800F00C00082840F09E80012D27D090
:102990007068E16900F480028A4221D1216A00F066
:1029A0003F028A421CD147F6C071626A0140B1EB16
:1029B000821F15D1A26A0023CFF6FF7303EBC23248
:1029C00000F440316FF30F02914209D1E16A00F047
:1029D0007060B0EB016F03D1002002B0BDE8F08160
:1029E000012002B0BDE8F0816069002840F20000DB
:1029F000C4F2472057D00121C0F8801EFFF7A6FD82
:102A0000054600BF706F8007B5D4FFF79FFD401BE0
:102A10000228F7D9A6E0306C10F080580AD10020C7
:102A20000190306C40F080503064306C00F0805089
:102A30000190019847F20007C4F200073868C0050A
:102A400024D4386840F480703860FFF77FFD054675
:102A50003868C0051AD4FFF779FD401B0228F7D962
:102A600080E0E068002851D00020C4F24720012116
:102A70000160FFF76BFD0546306880073FF571AFD9
:102A8000FFF764FD401B0228F6D96BE0A568052D11
:102A900050D0012D52D0306F20F001003067306FE0
:102AA00020F004004DE00021C0F8801EFFF74EFD2D
:102AB000054600BF706F80077FF55DAFFFF746FDED
:102AC000401B0228F6D94DE00027C4F2472700201A
:102AD0003866FFF73BFD022D05460BD130688001BB
:102AE00058D5FFF733FD401B02284FF00300F5D9FE
:102AF00073E700BF306880017FF56EAFFFF726FDFA
:102B0000401B02284FF00300F4D966E70020C4F20E
:102B1000472000210160FFF719FD05463068800756
:102B20007FF526AFFFF712FD401B02284FF0030090
:102B3000F4D952E7306F40F004003067306F40F056
:102B400001003067FFF702FD002D054641F288378E
:102B500014D000BF306F800713D4FFF7F7FC401B81
:102B6000B842F7D9032002B0BDE8F081FFF7EEFCD0
:102B7000401BB8424FF003003FF62FAF306F800785
:102B8000F4D4B8F1000F7FF4F9AE306C20F080502F
:102B90003064F3E604F11C052FCD08430021CFF685
:102BA000FF7140EA821001EBC3316FF30F0140EA7D
:102BB00005600843706001203866FFF7C7FC0446D3
:102BC000306880013FF508AFFFF7C0FC001B02280A
:102BD0004FF00300F4D900E780B501F0C5FC80BDDB
:102BE0007047000080B501F0BFFE032808BF80BD1C
:102BF00040F2EC1100EBC000C2F2000101EB8000DA
:102C00000069002818BF804780BD0000002804BF6D
:102C10000120704710B5044690F8410028B9002003
:102C200084F84000204600F021F8242084F8410078
:102C30002068C16821F40051C160204601F0A4FE63
:102C40002068016921F490410161416921F02A0164
:102C50004161C16841F40051C160002020216064DD
:102C600084F8411084F84210606310BD70B586B0DE
:102C70000446006841F20041C4F201010026884286
:102C8000CDE90466CDE9026601964ED044F6000116
:102C9000C4F20001884240F09580002643F63000DF
:102CA0000096C4F20200016941F4802101610169CA
:102CB00001F48021009100990096016841F004011F
:102CC0000160006801A900F00400009000984FF432
:102CD000406001900220CDE9020603200490072005
:102CE000059040F60000C4F20200FFF761FB40F2DD
:102CF000DC2546F22800C2F20005C4F202004FF0C3
:102D000000614FF4806285E843002846C5E903620C
:102D1000C5E90566C5E907666E62FFF7AFFA0028E8
:102D200018BFFEF709FDE56349E043F63000009661
:102D3000C4F20200416941F020014161416901F0A2
:102D40002001009100990096016841F04001016066
:102D5000006801A900F04000009000984FF4844002
:102D600001900220CDE9020603200490082005907E
:102D700040F60000C4F2020000F58050FFF718FB97
:102D800046F22800C4F2020040F23C3500F58F60A4
:102D9000C2F200054FF0206140224FF4806385E8C5
:102DA00047002846C5E90436C5E90666C5E9086650
:102DB000FFF764FA002818BFFEF7BEFCA56305F113
:102DC0003800046006B070BD80B590F84230202B0A
:102DD0001CBF022080BD00294FF0010318BF002A4C
:102DE00001D1184680BD0023036301F03BFE03467A
:102DF000184680BD80B501F0B7FD032808BF80BD2F
:102E000040F2EC1100EBC000C2F2000101EB8000C7
:102E1000C068002818BF804780BD000080B501F061
:102E2000A3FD032808BF80BD40F2EC1100EBC000F9
:102E3000C2F2000101EB80008068002818BF8047C3
:102E400080BD0000FEE7000010B52DED088B88B3B3
:102E5000B0EE408A90ED010A90ED069A90ED021ACC
:102E600090ED07AA29EE000A38EE400A2AEE011A70
:102E700030EE41BA04461BEE100A01F05BFE00285A
:102E800008BFB0EE4B8A94ED030A94ED041A94ED5A
:102E9000052A20EE080A29EE011A30EE010A2AEE70
:102EA000021A30EE010A84ED068A84ED079ABDEC21
:102EB000088B10BD9FED020ABDEC088B10BD00BF52
:102EC00000000000002808BF704710B5F5EE400A6A
:102ED0000446C0ED000A0020F1EE10FAA061E061A6
:102EE0002EDD80EE200A9FED1E1A81EE000A04F00E
:102EF000E3FC9FED1C1AB7EE002A20EE011A31EE1A
:102F0000023A20EE000ABFEE005A30EE033A30EEED
:102F1000055A32EE411A80EE034A35EE055A30EE7C
:102F2000010A85EE035A80EE030A34EE041A84ED9A
:102F3000034A84ED041A84ED054A84ED015A07E042
:102F40004FF07E519FED050AC4E903106061606097
:102F500084ED020ABDE81040704700BF0000000089
:102F6000DB0F4940F304B53F10B52DED048B10B3D2
:102F7000B0EE408A90ED030A90ED041A90ED052A18
:102F800030EE010A30EE020A88EE009A044619EE8D
:102F9000100A01F0BFFD00282046B0EE480A08BF25
:102FA000B0EE489A84ED069A84ED079AFFF74CFF3D
:102FB000BDEC048B10BD9FED020ABDEC048B10BD6F
:102FC00000000000B0B5012802D9FF2040B2B0BD1A
:102FD00040F26425C2F20005044655F8200060B9AD
:102FE0004820FDF76FFE002845F82400EDD0482169
:102FF000FDF731FA55F824000470002040B2B0BD4E
:10300000B0B584B048B304780546204600F064F8B3
:1030100028B36988A1F201210A295BD8012202FAAA
:1030200001F10A071DD111F0F00F30D040F2FF116D
:10303000009108218DF804100A3000216A4600BF73
:1030400000EB41035B7802EB41056B7110F8113026
:1030500001310429AB71F3D131E0FE2037E0FC20CF
:1030600035E04FF40071009108218DF80410023012
:1030700000216A4600EB41035B7802EB41056B716E
:1030800010F8113001310429AB71F3D117E040F28F
:10309000FF21009108218DF80410123000216A46AA
:1030A00000EB41035B7802EB41056B7110F81130C6
:1030B00001310329AB71F3D10020ADF80B00694653
:1030C0002046FDF71BFD002818BF4FF0FF3040B22F
:1030D00004B0B0BDFF20FAE701288FBF002040F206
:1030E0006421C2F2000151F82000704748B1022863
:1030F0000BD0012814BF4FF6FF704FF4804000B290
:10310000704742F2107000B2704747F2305000B280
:1031100070470000022905D2A0F2012189B20629D8
:1031200009D805E007D1A0F2052189B2052902D806
:10313000013840B27047FF2040B27047F0B581B00F
:1031400008B307460078FFF7C7FFE0B1014690F8E3
:103150004400C0B101F11802002306E0012585B149
:1031600091F844500133AB420DD252F82340002C69
:10317000F4D065887E88B542F0D100252046002D28
:10318000EED101B0F0BD002001B0F0BD022884BF37
:10319000B7EE000A704740B202A101EB800090ED4B
:1031A000000A704700001042000098410000803F74
:1031B00070B538B104460078FFF704FF28B1FF204E
:1031C00040B270BDFE2040B270BD2078FFF784FF92
:1031D0000028F4D090F8442005469AB105F1180073
:1031E000002104E095F84420013191420AD250F8C0
:1031F0002120002AF6D0528863889A42F2D1FD201D
:1032000040B270BD0A2ADAD85020FDF75BFD0028D5
:10321000D5D0064620686168C6E9000106F11800AD
:103220002821FDF718F962792078618886F828202E
:103230000322FDF71DFB18B13046FDF73FFDBEE749
:1032400095F8440005EB8001013085F8440000202A
:1032500040B28E6170BD000080B59FED020A00F0A3
:1032600003F880BD0000000070B52DED048B002830
:103270003ED005460078B0EE408AFFF72DFFC8B378
:10328000B7EE000AB4EE408AF1EE10FAC8BFB0EE15
:10329000408ABFEE000AB4EE408A0446F1EE10FA0E
:1032A000B8BFB0EE408A6879B1EE489A0028284647
:1032B00008BFB0EE489AFFF741FFE8B12E79688861
:1032C0003146FFF727FF002818D405463046FFF7A0
:1032D0000DFF00EE100AB8EEC00A29EE000ABDEE9E
:1032E000C00A10EE100A04EB45014880002006E0F9
:1032F000FE2004E0FC2002E0FC2000E0FF2040B2C1
:10330000BDEC048B70BD00002DE9F04F87B00028A4
:1033100052D004460078FFF7DFFE00284ED0054665
:1033200090F8440000284BD005F11806E8464FF00D
:10333000010A40F2E93B4FF0000908E001210029B1
:1033400041D095F8441009F1010989453AD256F85F
:103350002970002FF2D07A8861888A42EED12078D5
:1033600042460023FDF77EF970B1FDF7AFFCD7E9C7
:103370000823801A9941B0EB0B0071F1000016D3BD
:1033800000203876FC2013E087F818A0FDF79EFC9B
:10339000C7E908013846414600F022F907F1080361
:1033A0000FCB07F12C0C8CE80F00002000E0FF2071
:1033B00000210029C5D106E0FE2004E0FC2002E047
:1033C000FC2000E0FC2040B207B0BDE8F08F000018
:1033D00080B540F28C2046F20041C2F20000C4F2F7
:1033E00000010322002380E80E0000F10C014FF4DD
:1033F000102C4FF4001E81E8085083618383FEF790
:1034000053FC002818BFFEF797F980BD80B540F245
:10341000B42046F60001C2F20000C4F2000103220B
:10342000002380E80E0000F10C014FF4102C4FF443
:10343000001E81E8085083618383FEF735FC002875
:1034400018BFFEF779F980BD80B582B0002043F641
:1034500030010190C4F202010A6842F400120A60CD
:103460000A6802F400120192019A00900868002292
:1034700040F4800008600868052100F48000009096
:1034800000980C20FFF7E2F80C20FFF7DBF845204E
:1034900005210022FFF7DAF84520FFF7D3F802B044
:1034A00080BD000080B544F25D5048F2AC02C0F629
:1034B0000000C0F60002002101F09EFE40F28821CB
:1034C000C2F20001086044F2656048F24002C0F6B2
:1034D0000000C0F60002002101F08EFE80BD000059
:1034E00081B0002143F630000091C4F2020002686E
:1034F00042F002020260026802F002020092009AA8
:103500000091026842F040020260026802F040024C
:103510000092009A0091026842F001020260026883
:1035200002F001020092009A0091026842F0080243
:103530000260026802F008020092009A009102689C
:1035400042F004020260026802F004020092009A53
:103550000091016841F080010160006800F0800086
:103560000090009801B0704780B540F29C3044F65E
:103570000001C2F20000C4F2000148F2A062002380
:103580004FF00C0CC0F2010280E80E00C0E90333DA
:10359000C0E905C3C361FFF739FB002818BFFEF778
:1035A000CBF880BD80B540F2E43041F20041C2F278
:1035B0000000C4F2010100234FF00C0C4FF4E13283
:1035C00080E80E00C0E90333C0E905C3C361FFF71B
:1035D0001DFB002818BFFEF7AFF880BDFEE7000016
:1035E0002DE9F0478846B1F80D10044608BA4FEAB5
:1035F0001049B8F811002679B8F80F1005BA30460E
:1036000091FAB1FAFFF772FD07463046FFF7BEFDAB
:1036100001EE109A9FED453AB8EE412A9FED441A0B
:1036200022EE032A22EE014A02EE10AA15FB27F031
:10363000B8EEC23A02EE100AA0799FED3E5AB8EEFB
:10364000C22A22EE052A48B1B4F84000A9EB0000D6
:10365000B0F5805F0CDD4FF0FF300DE00020A4F8E6
:103660004090C4E9110084ED024A84ED033A1CE065
:1036700010F5805F03DA0120616C0844606494ED0A
:10368000115A83EE003AB8EEC55A25EE015A34EECF
:10369000054A84EE004AA4F8409020EE022A84ED08
:1036A000033A84ED124A84ED024A94ED020A84ED55
:1036B000042AB5EE400AF1EE10FA08DA30EE010AFB
:1036C000B5EE400AF1EE10FAF8DB84ED020A94ED53
:1036D000020AB4EE410AF1EE10FA0ADB9FED162A57
:1036E00030EE020AB4EE410AF1EE10FAF8DA84ED97
:1036F000020A94F8280078B131EE400A84ED020AFB
:1037000094ED030A94ED041AB1EE400A84ED030A25
:10371000B1EE410A84ED040A98F8130000EE100A95
:10372000B8EE400A84ED050ABDE8F08700000039D4
:10373000DB0FC94000008038DB0FC9C0FEE7000086
:1037400000F0070080F00703042B28BF04234FF08C
:10375000FF3C03380CFA03F338BF00209943814043
:103760000CFA00F022EA000008437047B0B52DEDD6
:103770000A8B044610EE100AB0EE618AB0EE419A50
:10378000B0EE60AAB0EE40BA01F0CCF9002800F02B
:103790009C801AEE100A01F0C5F9002800F095800F
:1037A00019EE100A01F0BEF9002800F08E8018EE24
:1037B000100A01F0B7F9002800F087806068B0EEC9
:1037C0004B0A90ED071AF0EE4A0AFDF739FD6068E2
:1037D000B0EE40BA90ED001A04F11C0020EE01CAD0
:1037E00021EE0A0AFFF730FB207888B1012811D1B9
:1037F00094ED051A94ED022A30EE411AB4EE428A95
:10380000F1EE10FAC8BFB0EE482A81EE029A01E04C
:103810009FED309A19EE100A84ED04BA84ED050A82
:1038200001F080F965689FED2B0A002808BFB0EE13
:10383000409A95ED010A95ED032A2CEE000A29EE37
:10384000022A95ED021A30EE42AA94ED030A9FED8A
:10385000229A2CEE082A32EE008AB4EE491AF1EED2
:1038600010FA28EE01BA1ADD18EE100A01F05AF922
:10387000A8B13AEE0B0A95ED051AB0EEC00AB4EE07
:10388000410AF1EE10FA0ADC95ED040AB0EEC81A0E
:10389000B4EE401AF1EE10FAD8BF84ED038A3AEE86
:1038A0000B8A18EE100A01F03DF970B1D5ED050A4A
:1038B000F4EE490AF1EE10FA05DDB0EE480AFCF725
:1038C0003DFEB0EE408A84ED068A94ED060ABDEC1A
:1038D0000A8BB0BD00000000BD37863570B52DEDF8
:1038E000048B90B3044650681646B0EE408A0D46ED
:1038F00001F018F958B3B06801F014F948B3F06852
:1039000001F010F938B3306901F00CF928B370698F
:1039100001F008F918B3B7EE000A80EE089A666065
:1039200019EE100A01F0FEF8D8B1D6ED060A04F13E
:103930001C00B0EE480A84ED029AFFF7C3FA204655
:10394000257000F013F800200CE0FF200AE0FF20B3
:1039500008E0FF2006E0FF2004E0FF2002E0FF2057
:1039600000E0FF2040B2BDEC048B70BD10B568B123
:1039700000F11C0100249FED070AC0E90344C0E9DF
:1039800005440846FFF7F0FA60B210BDFF2460B2AC
:1039900010BD00BF0000000000280EBFFF21002165
:1039A000C16048B270470000000000000000000045
:1039B000EFF30980BFF36F8F154B1A681EF0100FDD
:1039C00008BF20ED108A20E9F04F10602DE90900B2
:1039D0004FF0500080F31188BFF34F8FBFF36F8F0C
:1039E00002F06AFD4FF0000080F31188BDE8090085
:1039F00019680868B0E8F04F1EF0100F08BFB0EC6F
:103A0000108A80F30988BFF36F8F704700BF00BF33
:103A10002805002000000000000000000000000059
:103A2000074B19680868B0E8F04F80F30988BFF3C6
:103A30006F8F4FF0000080F31188704700BF00BF08
:103A40002805002080B501F0A7F880BD90ED000AA0
:103A500091ED001AB7EE002A30EE011AB4EE421AC8
:103A6000F1EE10FAD8BF704782EE011A20EE010A7B
:103A700080ED000A91ED000A21EE000A81ED000AB6
:103A800070470000B0B52DED048B10B30446B0F8BC
:103A9000A00000B394ED011A94ED272A9FED278A28
:103AA000D4ED1E0A94ED310A31EE429AB0EE481A76
:103AB0000D46FDF7C5FB6169B7EE001A91ED042ACA
:103AC00081EE022AB4EE429AF1EE10FA05DA0020F5
:103AD0002FE0FF202DE0FF202BE0B4EE410AF1EEB5
:103AE00010FA4FF0000024DCEA7812B3606804F1A9
:103AF000C405C4F89C0091ED030A2846B8EE400ABC
:103B000088EE000AF0EE480AFDF77CFB606990F849
:103B10003400012807D195ED000A9FED091A30EE17
:103B2000010A85ED000AB4F8A0000138A4F8A0004D
:103B3000002040B2BDEC048BB0BD00BFDB0FC9401C
:103B4000EBAB2B3CB0B52DED028B054600284FF0BA
:103B5000FF0026D00C4621B3FDF7B8F804F016FAA2
:103B60009FED128A00EE100A80EE080A85ED010A28
:103B7000FDF7ACF8D5E90223801A994104F006FA62
:103B800000EE100A80EE080A85ED040AFDF79EF8A3
:103B90002278C5E90201284621462A7000F034F94E
:103BA000002040B2BDEC028BB0BD00BF00247449C0
:103BB0002DE9F04F81B02DED028B044600284FF027
:103BC000FF0000F096800D46002900F09280B5EECF
:103BD000400AB0EE408AF1EE10FA40F38A802F7965
:103BE0006561BE003046FDF76DF8C4F8A4003046AC
:103BF000FDF768F8C4F8A8003046FDF763F8C4F88C
:103C0000AC003046FDF75EF8C4F8B0003801FDF7AF
:103C100059F820623046FDF755F8E0673046FDF769
:103C200051F8C4F88400C7EB071086003046FDF752
:103C300049F8C4F8C8003046FDF744F87E01C4F8DE
:103C4000CC003046FDF73EF8C4F848013046FDF799
:103C500039F8216AC4F84C01E1B1E16FD1B1D4F86F
:103C60008410B9B1D4F8A410A1B1D4F8A81089B1C6
:103C7000D4F8AC1071B1D4F8B01059B16169C96A07
:103C800041B1D4F8C81029B1D4F8CC10002918BF1C
:103C9000002834D1206AFDF711F8E06FFDF70EF827
:103CA000D4F88400FDF70AF8D4F8A400FDF706F86C
:103CB000D4F8A800FDF702F8D4F8AC00FCF7FEFF3A
:103CC000D4F8B000FCF7FAFF6069C06AFCF7F6FFB1
:103CD000D4F8C800FCF7F2FFD4F8CC00FCF7EEFFF4
:103CE000D4F84801FCF7EAFFD4F84C01FCF7E6FFF2
:103CF000FB2040B2BDEC028B01B0BDE8F08FD4F8E0
:103D000048010028C6D0FCF7EDFCDFB307EB8700C5
:103D100005F1380805F158094FEA400A4FF0000B49
:103D200000270026E86A3044FFF742FAD4F8C800BA
:103D300001215844B0EE480A4246FFF7CFFDD4F8BF
:103D4000CC0001215844B0EE480A4A46FFF7C6FDB0
:103D50006069D4F84811D0ED3E0AC819B0EE480A9F
:103D6000FFF7B0F86069D4F84C11D0ED3F0AC819DC
:103D7000B0EE480AFFF7A6F80A362037B2450BF135
:103D80003C0BCFD105F13000FFF712FA606990F8D3
:103D9000340078B1012835D104F1D00005F1B80222
:103DA0000121B0EE480AFFF799FD04F5867005F190
:103DB000D8020CE004F1D00005F178020121B0EE48
:103DC000480AFFF78BFD04F5867005F19802012182
:103DD000B0EE480AFFF782FD6069B0EE480AD0ED08
:103DE000400A04F5A870FFF76DF86069B0EE480A64
:103DF000D0ED410A04F5B870FFF764F80020C4E97B
:103E0000270076E7FC2074E7B0B500B304464069AC
:103E100090F82020F2B194F89820032A67D8DFE8C0
:103E200002F00259233A94ED0E0A9FED421A80EEF9
:103E3000010A90ED091AB4EE410AF1EE10FA68DDBC
:103E40006268012084F89800C4F8942061E0FF259E
:103E500068B2B0BD0025204684F8985084F8905090
:103E600000F00EF968B2B0BD90ED030A9FED2F1A75
:103E7000B8EE400A81EE000A94ED1E1A0020626836
:103E8000A4F8A000032084F89800C4F8942031EE30
:103E9000000A84ED310A204600F0F2F894ED010AA0
:103EA00094ED251A9FED222A30EE410AB4EE420A23
:103EB000F1EE10FA30DB94ED0E0A9FED1E1A00258C
:103EC00080EE010AB3EE041AB4EE410AF1EE10FAE4
:103ED000C8DA0DE094ED0E0A9FED161A80EE010A85
:103EE00090ED091AB4EE410AF1EE10FA04DA002559
:103EF00068B284F89850B0BD94ED010A94ED251A8B
:103F000090ED0A2A30EE410AB4EE420AF1EE10FAC0
:103F100005DA204600F0B4F8002568B2B0BD0120F3
:103F200084F89000022084F89800F5E7DB0FC9C000
:103F30009A99993E00007A4400284AD0F0B581B0A1
:103F40002DED028B04464069007920B3C0EB0010D0
:103F50009FED218A85000026002700BFD4F8C80005
:103F60003844FFF703FDD4F8CC003844FFF7FEFCDB
:103F7000D4F84801B0EE480A3044FEF7F5FFD4F813
:103F80004C01B0EE480A3044FEF7EEFF3C37BD422C
:103F900006F12006E2D104F1D000FFF7E7FC04F5BA
:103FA0008670FFF7E3FC9FED0C8A04F5A870B0EE75
:103FB000480AFEF7D9FF04F5B870B0EE480AFEF7DC
:103FC000D3FF0020BDEC028B01B0BDE8F04040B251
:103FD0007047FF2040B270470000000010B370B57A
:103FE00004464069007980B1C0EB001085000026CE
:103FF000D4F8C8003044FFF7CFFCD4F8CC003044EC
:10400000FFF7CAFC3C36B542F2D104F1D000FFF70D
:10401000C3FC04F58670FFF7BFFC0020BDE87040CC
:1040200040B27047FF2040B27047000020B310B587
:10403000416991F804C0BCF1000F14D0D0E92921E6
:10404000D0E92B430439A3F1040E231F043A0024C2
:1040500042F8044F41F8044F43F8044FBCF1010CFF
:104060004EF8044FF4D10021C0E92D11C0F8BC1066
:10407000BDE8104048B27047FF2148B270470000C9
:104080002DE9F04F81B02DED048B054600284FF04F
:10409000FF0000F038828946002900F03482686908
:1040A0002978047940F2324B0029C2F2000B00F06B
:1040B000D380287E002800F0E280022800F064818E
:1040C000012840F00982002C79D004EB84009FED98
:1040D000AC9A40F2342A9FEDAB8A4FEA400B6FF066
:1040E00003060024C2F2000A00274FF0000800BFB8
:1040F000686995ED300AC169C06A80EE091A007AD4
:10410000D5ED041A0138C0B201EB800090ED002A11
:10411000D5F8840022EE000A80EE090AD5F8C8100E
:1041200030448AED001AD0ED010A0819B0EE481AA1
:10413000FFF71CFBD5F8A410D5F884003144D5F85E
:10414000CC2081ED010A3044D5ED041A95ED220A08
:10415000D0ED010A1019B0EE481AFFF707FBD5E9B8
:1041600029203044011D80ED010A90190430FFF729
:104170006DFC05F1A40207CA304490ED010A8819CC
:1041800090ED011AD5F84C0130EE010A911938442E
:1041900081ED010AFEF758FE6969D5F8B000C96AD9
:1041A000304480ED010A01EB0800FFF75DF808F1EB
:1041B0000A0804362037C34504F13C0498D140F284
:1041C000E810C2F200009FEDDF8A90ED000AD5ED05
:1041D000041AD5ED1E0A05F1D000B0EE481AFFF71B
:1041E000C5FAD5ED041AD5ED230A05F58670B0EEB3
:1041F000481A85ED2D0AFFF7B9FA05F5B87085ED77
:104200002E0AFEF721FE686985ED2F0A3030FFF790
:104210002BF899F80200002800F07B8140F2324B25
:10422000C2F2000B9BF80000002840F0578199F87B
:104230000300002800F05281687E022103282976BD
:1042400000F07981022800F07181012814BF00205C
:104250000120A5F8A00041E164B104EB8400440012
:10426000002600BF6869C06A3044FEF7F5FF0A36D1
:10427000B442F7D168693030FEF7EEFF2EE1002C32
:1042800043D004EB84009FEDAF8A4FEA40086FF003
:10429000030600274FF0000A002400BFD5F8C8002D
:1042A0003844FFF779FBD5F88400D5F8C8103044BE
:1042B000D0ED010AD5ED041AC819B0EE480AB0EEE7
:1042C000481AFFF753FAD5F8A400D5F8AC10D5F882
:1042D0004C21304480ED010A881980ED010A02EB7F
:1042E0000A00FEF7B1FD6969D5F8B000C96A30442B
:1042F00080ED010A0819FEF7B7FF0A3404360AF107
:10430000200AA04507F13C07C8D140F2E810C2F2EC
:1043100000009FED8C8A90ED000AD5ED041AD5EDD2
:104320001E0A05F1D000B0EE481AFFF71FFAD5EDCE
:10433000041AD5ED230A05F58670B0EE481A85ED0E
:104340002D0AFFF713FA05F5B87085ED2E0AFEF772
:104350007BFD686985ED2F0A3030FEF785FF99F8FF
:104360000200002800F0BA802846FFF7E5FD284645
:10437000FFF734FE2846FFF759FE0120ADE000BFED
:1043800000C0DA450000000028464946FFF77AFBE6
:10439000002C6FD004EB84009FED699A9FED698A31
:1043A0004FEA40086FF0030400274FF0000A002690
:1043B000686995ED301AC16AC069097AD5ED041AA9
:1043C0000139C9B200EB810090ED000AD5F88400F4
:1043D00020EE010A80EE090AD5F8C8102044D0ED7D
:1043E000010AC819B0EE481AFFF7C0F9D5F8A410B1
:1043F000D5F884002144D5F8CC2081ED010A204471
:10440000D5ED041A95ED220AD0ED010AD019B0EECF
:10441000481AFFF7ABF9D5E929202044011D80EDAA
:10442000010A10190430FFF711FB05F1A40207CAB5
:10443000204490ED010A081990ED011AD5F84C01BD
:1044400030EE010A1119504481ED010AFEF7FCFC1F
:104450006969D5F8B000C96A204480ED010A88195D
:10446000FEF702FF0A3604340AF1200AB04507F1CC
:104470003C079DD19FED338AD5ED041AD5ED1E0A78
:1044800095ED310A05F1D000B0EE481AFFF76EF94C
:10449000D5ED041AD5ED230A05F58670B0EE481A5D
:1044A00085ED2D0AFFF762F905F5B87085ED2E0A46
:1044B000FEF7CAFC686985ED2F0A3030FEF7D4FE9E
:1044C00099F8030050B901202876A86F40F2E8114E
:1044D000C2F20001086001E0002028766869C06A25
:1044E000FEF78EFD68694168052903D3C06A28304C
:1044F000FEF786FD68693030FEF782FD99F803000B
:104500008BF80000002040B2BDEC048B01B0BDE888
:10451000F08F2846FFF710FD2846FFF787FD0020A3
:1045200040F2324B2876C2F2000BD7E76869406947
:10453000A5F8A000D2E741F60A20A5F8A000CDE733
:1045400000C0DA450000000000280FBFFF214176BF
:104550000021A0F8A01048B27047000080B500F01C
:1045600047FE00F0A3FE80BDB0B501380024B4EBD7
:10457000106F1CBF0120B0BD4EF21005CEF2000539
:1045800068604FF0FF300F2100F0F4FA0720AC60B4
:1045900028602046B0BD000080B5FDF7DDFF02F0C9
:1045A0008DFE012818BF02F05FF880BD70B592B093
:1045B00006AC20463021FBF74EFF002543F64000B5
:1045C0000595CDE90355CDE901550095C4F20200EA
:1045D0000168022641F080510160006800F08050BF
:1045E0000090009847F200000095C4F200000168B6
:1045F00041F480410160006800F480400090009820
:10460000012006904FF4803007904FF480000D9009
:1046100006200E90A820CDE90F0604201190204618
:104620000C96FEF735F988B90F20CDE901064FF455
:10463000A05004904FF48050059001A805210395E7
:10464000FEF718F8002804BF12B070BDFDF774F82B
:104650004EF68850CEF20000016841F4700101600E
:104660007047000010B500F061FB44F2617048F241
:104670008802C0F60000C0F60002002100F0BCFD78
:1046800040F6AC34C2F20004206044F2C96048F243
:104690006402C0F60000C0F60002002100F0ACFD8C
:1046A000606002200A21002200F0D6FBA0600320F7
:1046B0002821002200F0D0FBE06000F067FB00F052
:1046C00097FD00F0F3FD10BD00F018FB03F0F7FBC1
:1046D0009FED210B53EC102B03F06AFA03F0C2FBA1
:1046E0000446002000F0D6FA00F0FEFA40F2382826
:1046F000C2F2000805464046FCF72AFE40F26C294B
:10470000C2F200094846FCF78DFF2F1940F6C0158C
:1047100040F6AC36C2F20005C2F200060AE000BF65
:10472000F06829460022002300F0E6FB384600F03E
:10473000C1FA27440A20FCF783FF0028F0D048463E
:104740004146FCF729FE40462946FCF755FB484602
:10475000FCF768FFE4E700BF0000000000407F4076
:1047600000F0CCFA03F0ABFB9FED250B53EC102BC4
:1047700003F01EFA03F076FB8046002000F08AFA70
:1047800000F0B2FA0446FCF77FFDFCF777FD40F637
:10479000E815C2F200059FED1C0A01462846FFF706
:1047A00007FA28460221FFF7CFFE04EB080640F681
:1047B000AC3940F6843740F68034C2F20009C2F2C8
:1047C0000007C2F2000400BFD9F80C0039460022ED
:1047D000002300F0FDFAB88C79786080387869762B
:1047E00020702846FCF716FC28462146FFF7AAF958
:1047F000304600F05FFA4644E6E700BF00BF00BF66
:104800000000000000407F400000FA4310B5846BB8
:104810002068406994F84110212907D110F08000E8
:1048200004D00020E084204600F090F82068406921
:1048300094F84210222907D110F0400004D0002043
:10484000E085204600F05AF8606C40F0100060648B
:104850002046FEF7C7F910BD80B50168806B096876
:10486000C9052FD40021C185016851E8031F0268E2
:1048700021F4807142E80313002BF5D1016851E85F
:10488000051F026821F0010142E80513002BF5D154
:10489000016851E8051F026821F0400142E8051354
:1048A000002BF5D1202180F84210016B012909D19C
:1048B000016851E8031F026821F0100142E8031368
:1048C000002BF5D100214163016B012903D1818DBA
:1048D000FEF786F980BDFEF78DFA80BD80B5806B4E
:1048E00001214163016B012904D1818D4908FEF743
:1048F00077F980BDFEF792FA80BD0000016851E8AB
:10490000031F026821F4907142E80313002BF5D1D4
:10491000016851E8051F026821F0010142E8051312
:10492000002BF5D1016B01290AD100BF016851E8C4
:10493000031F026821F0100142E80313002BF5D198
:10494000202180F84210002101637047016851E87E
:10495000031F026821F0C00142E80313002BF5D1C8
:10496000202180F84110704744F600010068C4F22D
:10497000000101F54C420323904208BF0123401A75
:1049800018BF18467047000010B504460068D4E907
:1049900002C22369016921F4405111430161626936
:1049A00043EA0C01E3691143C268194349F20C63FD
:1049B0009A431143C1604169A26921F4407141F2F7
:1049C0000043114340F48062C4F201039A42416102
:1049D00002D1FDF717FF01E0FDF702FFE16963680F
:1049E0001922B1F5004FA0FB02011CD15A00DB0FC8
:1049F000FBF73AFC48F21F51C5F2EB11A0FB012373
:104A00005A096FF0630302FB0300322303EBC0007B
:104A1000A0FB01014FF4F87000EA111000EB021046
:104A2000C1F342111AE09A009B0FFBF71DFC48F2FC
:104A30001F51C5F2EB11A0FB01235A096FF063036C
:104A400002FB0300322303EB0010A0FB0101F02066
:104A500000EA511000EB0210C1F343112268084331
:104A6000906010BDF0B581B0134600270446816206
:104A700083854764222084F84200E06B44F65905A0
:104A800044F6DD060A462168C0F60005C0F60006B9
:104A9000C0E90F5644F60D06C0F600060431C0E921
:104AA0001367FDF753FC38B110206064202084F8B0
:104AB0004200012001B0F0BD00972068016800911C
:104AC000406800900098206950B100BF206850E80D
:104AD000030F216840F4807041E80302002AF5D1F9
:104AE000206850E8050F216840F0010041E8050208
:104AF000002AF5D1206850E8050F216840F04000F9
:104B000041E80502002AF5D1002001B0F0BD000007
:104B1000FEE7000000F0FF40B0F1FF4018BF0120A9
:104B20007047000000F0FF40B0F1FF4018BF0120C7
:104B30007047000020F00040A0F1FF40B0FA80F084
:104B400040097047002848BF704700F01F0101224C
:104B500002FA01F14EF200124009CEF2000242F8D0
:104B6000201070474EF60C50CEF200000068C0F3E3
:104B7000022070474EF6145300F00F02CEF20003ED
:104B800009011A4400F16043B0F1FF3FC8BF03F5CB
:104B900064421170704700004EF61F50CEF20000C4
:104BA00000210170704700004EF60C51CEF200015A
:104BB0000A684FF6FF031A4060F30A2242F0806051
:104BC00040F0FD7008607047F0B581B0F0B1044668
:104BD00040F22850C2F200000068A0421FD001F04D
:104BE0008BF940F23050C2F200006569076840F26C
:104BF0003850C2F20000066801F0A2F9BD424FF041
:104C0000020018BFB5420DD101B0F0BD4FF0500009
:104C100080F31188BFF36F8FBFF34F8FFEE7002043
:104C200001B0F0BD45F2A070C2F2000085420CD088
:104C300045F2B4710120C2F20001002D08BF04202A
:104C40008D4208BF042001B0F0BDA06A10B102205F
:104C500001B0F0BD94F858100320012908BF0220CC
:104C600001B0F0BDFDF786FCFFF7A0FCFEF738FCB5
:104C7000FEF7EAFBFEF7ACFBFEF7C8FBFEF774FCA1
:104C8000FEF790FC00F03EF8FEF70CFC00F064F834
:104C9000FEE70000EFF3058100291CBF6FF005005F
:104CA0007047002804BF0020704780B501F028FA43
:104CB000002080BD10B582B0EFF3058119B16FF00F
:104CC000050002B010BD044602F00CFB211A0129B8
:104CD000019005DB01A801F03DFA002002B010BDF3
:104CE0006FF0030002B010BD80B5EFF3058010B186
:104CF00002F0FEFA80BD02F0F5FA80BD4FF47A7042
:104D000070470000EFF3058000281CBF6FF005001E
:104D1000704740F2E410C2F200000168002911BFA0
:104D20004FF0FF30012101600020704780B5EFF3A4
:104D3000058000281CBF6FF0050080BD02F0BEFAA0
:104D400028B1022805D101F0AFFB002080BD012071
:104D500080BD4FF0FF3080BD10B5EFF30580002817
:104D60001CBF6FF0050010BD40F2E414C2F2000455
:104D7000206801281CBF4FF0FF3010BDFEF762FE17
:104D80000220206001F03EFB002010BD10B5EFF3C3
:104D9000058018B16FF00504204610BD02F08EFAB0
:104DA00002280ED080B902F07BFC01284FF00104EC
:104DB0000CD002F083FA002808BF4FF0FF342046E1
:104DC00010BD0024204610BD4FF0FF34204610BD1A
:104DD00010B582B01C46B0FA80F3B1FA81F25B09DB
:104DE0005209EFF3058CBCF1000F42EA030219D01F
:104DF000002C18BF0124224315D10022019201AAE0
:104E000001F036FF01281AD10198A8B14EF60450DE
:104E1000CEF200004FF080510160BFF34F8FBFF31F
:104E20006F8F09E01AB16FF0030002B010BD224687
:104E300001F05CFE012806D1002002B010BD6FF029
:104E4000020002B010BD6FF00100002C08BF6FF02F
:104E5000020002B010BD0000B0B582B014460029B7
:104E60004FF00005EFF3058218BF002802D1284655
:104E700002B0B0BD002AFAD19CB1A568D5B1E268F4
:104E8000502A16D32269A2B1D4F814C001FB00F253
:104E9000002394454FF0000228BF012210D24DB1EB
:104EA0000EE0012300226AB9E3B1002201F012FCF6
:104EB0000EE01DB9E2680AB92269C2B100220023DE
:104EC000002AF1D0A36822690025009501F026FC94
:104ED000054655B1002C14BF21680021284601F079
:104EE000D9F8C4E70025002DF4D10025BFE7626999
:104EF000B2FA82F25309D5E7B0B582B01C46B0FAD7
:104F000080F3B1FA81F5EFF305825B096D09002AA0
:104F100043EA050207D0002C18BF0124224306D023
:104F20006FF003052CE0CAB16FF0030528E0002202
:104F3000019201AA002301F04FFD01281CD1019824
:104F4000E8B14EF60450CEF200004FF080510160FF
:104F5000BFF34F8FBFF36F8F002511E02246002370
:104F6000002501F067FC01280AD06FF00105002C34
:104F700008BF6FF0020503E06FF0020500E00025B6
:104F8000284602B0B0BD000010B50C46EFF3058115
:104F900000291CBF6FF0050010BD014620F0010084
:104FA00050B111F001010AD1214601F0B7FE0128EC
:104FB00004BF002010BD09E06FF0030010BD2146C2
:104FC00001F090FF012804BF002010BD6FF0010028
:104FD000002C08BF6FF0020010BD000070B5EFF3A9
:104FE0000581B9B90028044614BF60680020010794
:104FF00010D494B1A36843B1E26800214F2A4FF066
:10500000000288BF01220AD84BB9E168B1FA81F1E8
:10501000490903E00025284670BD0121002200F067
:1050200001063AB1A168002E0CBF0120042001F056
:105030003FFB06E0C9B1002E0CBF0120042001F0A7
:105040002BFB054635B1002C14BF216800212846F2
:1050500001F020F8B5FA85F0400986F00101084317
:1050600008BF45F00105284670BD0025002DEAD196
:10507000F0E7000080B5EFF3058100291CBF6FF059
:10508000050080BD014620F0010040B111F0010192
:1050900008D100210022002301F0CCFB04E06FF0D6
:1050A000030080BD01F000FD013818BF6FF0020061
:1050B00080BD0000B0B584B048B3B1F1FF3F26DD3C
:1050C00004464FF0FF300390EFF3058018B300253E
:1050D0000DF1080C2046012200230295CDF800C0F6
:1050E00002F050F803AB204600210022009502F0A8
:1050F00049F80298D0B14EF60450CEF200004FF0BD
:1051000080510160BFF34F8FBFF36F8F0EE06FF0E0
:10511000030003900AE020460122002301F0B4FFBF
:1051200003AB20460021002201F0AEFF039804B03B
:10513000B0BD00002DE9F04F83B00C46EFF30581C0
:1051400029B16FF00507384603B0BDE8F08F05467A
:10515000002849D44FF0000B9246A00758BFAB4639
:1051600002F0C0F800906FF0010804F0010054460E
:105170000027BAF1000F08BF6FF00208019002E0AB
:105180004746002EDFD00020594602AA234602F0EF
:1051900063F906460128F3D1029807EA050140EABF
:1051A00001090198002809EA050007D100286FF0DD
:1051B000020718BF4F4607D0C5E700BFA8426FF0EF
:1051C000020708BF4F46BED0BAF1000FBBD002F0B5
:1051D00089F800994F46401A241A4FF0000038BF52
:1051E0000446002ECFD1AEE76FF00307ABE7000017
:1051F00080B502F05DF880BD70B584B08E460021A8
:1052000000280391EFF3058146D0002944D1FAB17B
:105210009369002B08BF1823382B16D81179C907BA
:1052200013D15569946811684FEA950C002D08BF99
:105230004FF0800CFCB1D6685C2E1BD3D5B115693C
:10524000C5B10024012555B91BE0002004B070BD94
:105250000124002118234FF0800C00258DB19468A3
:1052600012690294CDE900326246734601F0D0FE25
:10527000039011E00CB9D4689CB100250024002DE6
:10528000EDD14CB103AC00931FFA8CF2734601943C
:1052900001F08AFE012802D1039804B070BD0020FD
:1052A000E6E71469B4FA84F46409D6E710B5EFF3BD
:1052B000058100291CBF6FF0050010BD044660B1D8
:1052C0002046FFF781FC042804BF6FF0020010BDE8
:1052D000204600F093FF002010BD6FF0030010BDCA
:1052E000F0B581B00D4645F2C87140F22856C2F2C1
:1052F0000001C2F200060F6831680446081D00F084
:1053000087FD601C0AD14DB13068011D45F2A070C7
:10531000C2F2000000F0D8FD01B0F0BD3068E41921
:1053200044600AD340F23850C2F20000006831688D
:10533000043100F0ABFD01B0F0BD40F23050C2F2DC
:10534000000000683168043100F0A0FD45F22C70C7
:10535000C2F2000001688C4238BF046001B0F0BDA9
:1053600070B5044600F0C8FD45F20000C2F200002E
:10537000016840F2285501310160C2F20005296838
:1053800045F29476C2F2000641B1306860B92868EF
:10539000E16AC06A884298BF2C6005E02C60006812
:1053A000012801D100F0DEF945F20C00C2F2000044
:1053B000016801310160616445F21001C2F200012F
:1053C000E06A0A68904288BF086040F2405100EBF2
:1053D0008000C2F2000101EB8000211D00F074FD8D
:1053E00000F0AEFD306880B12868E16AC06A88428A
:1053F00028BF70BD4EF60450CEF200004FF0805131
:105400000160BFF34F8FBFF36F8F70BD70B582B077
:1054100000F072FD45F2CC76C2F20006306850BB57
:1054200045F2CC64C2F20004204600F01FFD45F2B4
:10543000E065C2F20005284600F018FD40F22C504D
:10544000C2F20000046040F23C50C2F2000040F2A0
:10545000334240F2D44305600025C2F20002C2F29A
:1054600000030A201021009501F058F9306010B1B6
:1054700003A100F00FFE00F063FD02B070BD00BF9D
:10548000546D725100000000F0B581B045F2040582
:10549000C2F200052868E0B145F2B47645F2000793
:1054A000C2F20006C2F2000700F026FDF068C468F0
:1054B000201D00F0ADFC38680138386028680138DC
:1054C000286000F03DFD204600F058F828680028CC
:1054D000EAD101B0F0BD000080B5026C002A08BF1F
:1054E00080BDD0E902C31344C360634524BF036891
:1054F000C360C36808461946FAF72EFF80BD000056
:1055000070B5866B036C0446E3B115461AB3E068C8
:105510001A46FAF721FFE168206C2268091A9142C5
:10552000E16003D2A16840420844E060A81EB0FADE
:1055300080F040093146002E18BF01210840361A7C
:10554000002516E02068002598B9A06801F0CCFF7E
:10555000A56005460DE060681A46FAF7FDFE216C6D
:10556000D4E90102002508446060904224BF20680D
:105570006060711C2846A16370BD000010B5044630
:1055800090F85900022808BF10BD012803D030B997
:10559000206B00F0EDFC204600F0EAFC10BD4FF05F
:1055A000500080F31188BFF36F8FBFF34F8F00BFA0
:1055B000FEE70000416A00290FBF0020006B006871
:1055C000C0F138007047000040F22C51C2F20001D7
:1055D00009680A68B2FA82F35B090360002A0EBF09
:1055E0000020C8680068704741F2F430C2F2000041
:1055F000C21D22F0070210F0070CA0EB020318BF37
:10560000104645F29872C2F200020021C2E9000180
:105610004FF47052BCF1000F18BF03F570520244F2
:10562000083A40F2345322F00702C2F200031A6033
:10563000C2E90011111A1A68C0E9002145F2287068
:10564000C2F20000016045F22070C2F20000016069
:1056500045F2F460C2F200000121017070470000C1
:1056600040F240544EF60455C2F20004CEF200055A
:105670004FF08056FFF708FF20680228FAD32E600B
:10568000BFF34F8FBFF36F8FF4E70000002808BF10
:10569000704780B500210160C0E90211002100229D
:1056A000002301F0C7F8BDE880407047B0B5049D05
:1056B000002914BF2A602D60C5E90F012846012189
:1056C0001C4601F077F885F84C40B0BD2DE9F04755
:1056D0000A9C8246206B16460F46DDE90859910068
:1056E000A5229846FAF7AFFE206B00EB8600A0F1EA
:1056F000040020F007067FB104F13400002100BF50
:105700007A5C42547A5C1AB10F2901F10101F7D396
:10571000002084F8430002E0002084F834000027D1
:10572000201D372D28BF3725E562C4E9135700F047
:10573000A9FB04F1180000F0A5FBC5F13800A06139
:1057400030465146424624616462676584F8587069
:1057500000F04AFBB9F1000F206018BFC9F8004003
:10576000BDE8F087B0B540F240550024C2F2000514
:10577000281900F07BFB1434B4F58C6FF8D145F296
:10578000F864C2F20004204600F070FB45F20C758C
:10579000C2F20005284600F069FB45F24070C2F2F3
:1057A000000000F063FB45F2B470C2F2000000F0AC
:1057B0005DFB45F2A070C2F2000000F057FB40F222
:1057C0003050C2F20000046040F23850C2F20000D3
:1057D0000560B0BD80B545F29872C2F2000200BF0C
:1057E000114612688242FBD3D1F804C001EB0C03CE
:1057F000834203D14068604448600846D0F804C042
:1058000000EB0C03934201D013460BE040F23453FB
:10581000C2F200031B689A4204D0D2E9003E0EEBAC
:105820000C0242608142036018BF086080BD000026
:1058300080B58C46014641F804CF9445006108D9F3
:105840009A4201D29C4511D240F22C50C2F2000083
:1058500007E08069D21A824208D240F23C50C2F27C
:105860000000006800F012FB002080BD012080BD18
:1058700010B5044600F040FBA06BB0FA80F044097C
:1058800000F05EFB204610BD10B5044600F034FB6E
:10589000A06BE16B401AB0FA80F0440900F050FBB5
:1058A000204610BD08480068006880F308884FF063
:1058B000000080F3148862B661B6BFF34F8FBFF368
:1058C0006F8F00DF00BF00BF08ED00E070B582B051
:1058D00040F22C52C2F2000212680546D2680E460F
:1058E000D468201D00F094FA94F82800410704D4ED
:1058F00000F0FE0084F8280010E0A069324641194B
:1059000020462B46FFF794FF40B100262046002199
:105910002A460023009601F087FF20B1216A204625
:10592000884702B070BD4FF0500080F31188BFF37C
:105930006F8FBFF34F8F00BFFEE700002DE9F041EE
:1059400086B045F2CC77C2F20007386802A900227F
:105950004FF0000801F0CAF800286AD001AC02AD8F
:105960000BE000F0FE0086F8280000BF38682946EA
:10597000002201F0BBF800285BD00298B0F1FF3F95
:1059800003DCDDE903200599904702980028EDD457
:10599000049E706910B1301D00F03AFA204600F004
:1059A000B3F802990929E1D80246DFE801F00808B6
:1059B00008052A390808052A96F82800D1E796F83C
:1059C0002800039BB16940F0010086F828001944C3
:1059D0003046FFF72DFF0028C8D0316A304688478F
:1059E00096F828004007C1D50398B16900230A182A
:1059F00030460021CDF8008001F016FF0028B5D117
:105A000023E096F8280040F00101039886F828105A
:105A1000B06188B1811830461346FFF709FFA5E74A
:105A200096F8280081073FF59CAF304600F0A0FAB9
:105A30009CE706B0BDE8F0814FF0500080F311887C
:105A4000BFF36F8FBFF34F8FFEE74FF0500080F32F
:105A50001188BFF36F8FBFF34F8F00BFFEE70000C9
:105A600070B582B00E46044600F01EFD01A800F09D
:105A70004BF8019919B101F013FE02B070BD054653
:105A80004EB9A54207D301F00BFE20462946FFF789
:105A90001DFF02B070BD4EB140F23C50C2F200009A
:105AA00000680068B0FA80F0420900E0002245F288
:105AB000CC70C2F200000068611B00F0FFFA01F038
:105AC000EFFD0028D9D14EF60450CEF200004FF081
:105AD00080510160BFF34F8FBFF36F8F02B070BD75
:105AE00040F23050C2F200000168096821B100683C
:105AF000C068C068406801E04FF0FF3045F22C718B
:105B0000C2F200010860704770B5044601F0EAFB7C
:105B100040F22456C2F2000631680546884203D29C
:105B200000F008F8012000E00020206028463560E1
:105B300070BD00002DE9F04182B040F22C57C2F256
:105B400000073868016891B34FF0000809E000BF12
:105B5000606038682946246100F098F93868016867
:105B600029B3C068C4680668251D284600F050F9AE
:105B7000216A2046884794F828004007EED5A0699E
:105B80003044B042E4D82046002132460023CDF80C
:105B9000008001F049FE0028E0D14FF0500080F372
:105BA0001188BFF36F8FBFF34F8F00BFFEE740F246
:105BB0003C51C2F200010A6808603A6002B0BDE8D8
:105BC000F081000081B00020009040F21410C2F279
:105BD000000000684FF0500181F31188BFF36F8F10
:105BE000BFF34F8F013001D0FEE700BF00980028BF
:105BF000FCD001B07047000082B001AC2046FFF736
:105C0000E3FC0199FFF72CFFFFF798FEF6E7000091
:105C1000F0B581B0044600F06FF994F94560012EAB
:105C20000FDB04F1240500BF286850B1284601F0BD
:105C3000EFFC002818BF00F051FB70B2013E0128B4
:105C4000F2DCFF2684F8456000F07AF900F054F9A0
:105C500094F94470012F0EDB04F11005286850B14F
:105C6000284601F0D5FC002818BF00F037FB78B2B9
:105C7000013F0128F2DC84F8446000F061F901B0D2
:105C8000F0BD00002DE9F04381B0044600F00CFCAB
:105C900040F23456C2F200063068002808BFFFF711
:105CA000A3FC45F2F468C2F2000898F8000000284E
:105CB00018BF4FF0004020420DD0002401F0F0FC4E
:105CC00060071ED04FF0500080F31188BFF36F8F34
:105CD000BFF34F8FFEE7C4B114F0070004F10801D1
:105CE0001EBF081A00F108015FEA41700ED04FF0A4
:105CF000500080F31188BFF36F8FBFF34F8F00BF49
:105D0000FEE7204601B0BDE8F083002145F220798E
:105D1000C2F20009D9F800004A1E8242CDD245F2F3
:105D20009870C2F2000005682F4657F8042F8A4287
:105D300011D22B685BB100BF1F4657F8042F2846CD
:105D40001D468A4207D22B68002BF5D103E045F2AD
:105D50009870C2F2000033689D42AED004682B6890
:105D6000521A112A036010D36818430709D04FF064
:105D7000500080F31188BFF36F8FBFF34F8F00BFC8
:105D8000FEE742603960FFF725FD45F2287039686B
:105D9000D9F80020C2F200000368511A9942C9F8EC
:105DA000001038BF016098F80000396800284FF0F3
:105DB000000018BF41F00041286045F23470C2F283
:105DC0000000026808343960511C016076E7000069
:105DD00040F22850C2F20000016819B101680A6D52
:105DE00001320A6500687047034645F6C530C0F6C3
:105DF00000004FF0807C21F0010103E903106FF0F7
:105E0000020043F8240CA3F1440043F8202C70470F
:105E1000D0E9013201699A60D1F804C082688445F2
:105E2000536008BF4A6000220261086801380860B8
:105E30000868704745F21423C2F20003036045F27C
:105E40001400C2F20000086080201060704700005B
:105E500045F27063C2F20003036045F27020C2F2A3
:105E6000000008604FF48070106070474FF0FF3101
:105E7000024642F8081F00214260C0E90322016087
:105E800070470000002101617047000080B5D1F823
:105E900000C01CF1010207D000F108039E465B68B8
:105EA0001A686245FAD901E0D0F810E0DEF8042063
:105EB00008614A609160C1F808E0CEF804100168FA
:105EC0000131016080BD0000D0F800C04368086166
:105ED0009A684B608A609A68996051600CF1010180
:105EE00001607047DFF80C00016841F47001016047
:105EF000704700BF88ED00E04FF0500080F311883C
:105F0000BFF36F8FBFF34F8F40F21410C2F2000047
:105F100001684A1C026001B170474EF60450CEF28F
:105F200000000068000608BF70474FF0500080F383
:105F30001188BFF36F8FBFF34F8F00BFFEE70000E4
:105F400040F21410C2F20000016839B10139016059
:105F500018BF7047002080F3118870474FF0500041
:105F600080F31188BFF36F8FBFF34F8FFEE7000000
:105F7000B0B5002808BFB0BD044645F2F460C2F2D7
:105F80000000007854F8041C002818BF4FF00040AF
:105F900008420CD0A4F108052A6892B14FF05000D5
:105FA00080F31188BFF36F8FBFF34F8FFEE74FF081
:105FB000500080F31188BFF36F8FBFF34F8F00BF86
:105FC000FEE721EA000044F8040C00F06DFA45F207
:105FD0002071C2F2000154F8040C0A6810440860F1
:105FE0002846FFF7F7FB45F23870C2F2000001685F
:105FF0000131016001F054FBB0BD00004EF2100011
:10600000CEF2000000210160816040F20001C2F286
:106010000001096844F6D352C1F26202A1FB0212E8
:106020004FF0FF3101EB9211416007210160704791
:10603000EFF30580102814D34EF2F031CEF20001B8
:10604000405C44F6F471C2F200010978884208D23B
:106050004FF0500080F31188BFF36F8FBFF34F8F65
:10606000FEE74EF60C50CEF2000044F6F8710068E0
:10607000C2F20001096800F4E060884298BF7047EE
:106080004FF0500080F31188BFF36F8FBFF34F8F35
:10609000FEE7000045F2547C0022C2F2000C00BF73
:1060A0005CF8323023B10132082A08BF7047F7E7A5
:1060B0000CEBC2034CF832105860704770B51546AF
:1060C0000E460446FFF718FF94F84400FF2804BF6B
:1060D000002084F8440094F84500FF2804BF002005
:1060E00084F84500FFF72CFFA06B28B904F12400C9
:1060F00031462A4600F014F92046FFF789FD70BDAD
:1061000010B5D8B1044645F20800C2F2000000689C
:1061100048B14FF0500080F31188BFF36F8FBFF389
:106120004F8F00BFFEE700F0BFF920460021FFF7C8
:10613000D7F801F0B5FA002818BF10BD4EF604508C
:10614000CEF200004FF080510160BFF34F8FBFF3DC
:106150006F8F10BDB0B590B10D46D1B1044645F278
:106160000800C2F200000068E8B14FF0500080F370
:106170001188BFF36F8FBFF34F8F00BFFEE74FF063
:10618000500080F31188BFF36F8FBFF34F8F00BFB4
:10619000FEE74FF0500080F31188BFF36F8FBFF31D
:1061A0004F8F00BFFEE700F07FF945F2C870C2F2E2
:1061B000000000682268904202EB050102D2914281
:1061C00002D309E0914201D3814205D92160081A26
:1061D0000021FFF785F800E0216001F061FA002856
:1061E00018BFB0BD4EF60450CEF200004FF0805103
:1061F0000160BFF34F8FBFF36F8FB0BD70B5044622
:10620000FFF77AFE40F22856002CC2F2000608BFC3
:106210003468251D2846FFF7FBFDA06A18B104F17C
:106220001800FFF7F5FD45F20C00C2F2000001680E
:1062300001310160306884420CD045F20000C2F2A6
:1062400000000168013901602046FFF797F9FFF768
:1062500047FC0DE045F2B470C2F200002946FFF79A
:1062600033FE45F20400C2F2000001680131016012
:10627000FFF766FE45F29470C2F200000068E8B1D4
:106280003068844218BF70BD45F20800C2F20000B9
:10629000006840B14FF0500080F31188BFF36F8F5A
:1062A000BFF34F8FFEE74EF60450CEF200004FF0E2
:1062B00080510160BFF34F8FBFF36F8F70BD00003F
:1062C00045F23071C2F200010968016045F2C871FF
:1062D000C2F20001096841607047000045F2D470C5
:1062E000C2F20000012101607047000010B568B1E2
:1062F0000C4640F22851C2F2000109681831FFF73C
:10630000C5FD20460121FEF7EBFF10BD4FF0500008
:1063100080F31188BFF36F8FBFF34F8FFEE700004C
:10632000B0B590B10D4640F22851C2F200010968A3
:1063300014461831FFF7C8FD002C18BF4FF0FF3589
:1063400028462146FEF7CCFFB0BD4FF0500080F349
:106350001188BFF36F8FBFF34F8F00BFFEE70000C0
:1063600070B528B3026D04461AB3E06C884238BF9A
:106370000846012A1CD1E16A814208BF70BD40F283
:106380002852C2F200021268A2421CD0A269E06246
:10639000002A5CBFC0F13800A06140F2405660693D
:1063A00001EB8101C2F2000606EB8101884214D0A4
:1063B00070BD4FF0500080F31188BFF36F8FBFF3B3
:1063C0004F8F00BFFEE74FF0500080F31188BFF3FE
:1063D0006F8FBFF34F8F00BFFEE7251D2846FFF7E5
:1063E00017FD45F21001C2F20001E06A0A6890420E
:1063F00088BF086000EB800006EB80002946FFF7AD
:1064000063FD70BD10B586B0002405A804A903AAD9
:10641000CDE90444FFF70EFDDDE9032005990023D3
:10642000CDE9010145F26160C0F600001CA10094B5
:1064300000F0EEFD45F22471C2F20001086010B1D7
:1064400001F0B8F90446601C20D0012C1CD14FF09B
:10645000500080F31188BFF36F8FBFF34F8F45F269
:106460002C70C2F200004FF0FF31016045F29470D1
:10647000C2F200000121016045F2C870C2F20000C2
:106480000021016000F066F806B010BD4FF050002A
:1064900080F31188BFF36F8FBFF34F8FFEE700BF0C
:1064A00049444C450000000045F20800C2F20000DB
:1064B000016801310160704745F20800C2F2000036
:1064C000006830B145F2D470C2F2000001210160D1
:1064D000704745F2D470C2F20000002145F2100C62
:1064E0000160C2F2000CDCF8001040F2405201EBF7
:1064F0008103C2F2000252F8230048B902EB830084
:10650000A0F11403D9B153F8140901390028F9D0C6
:1065100001EB810002EB800252F8040F4368101D6A
:106520008342136001D158681060106840F228520D
:10653000C068C2F200021060CCF8001070474FF043
:10654000500080F31188BFF36F8FBFF34F8F00BFF0
:10655000FEE7000080B582B04EF20040CEF20000AF
:106560004CF27021C4F20F11D0F800294B1C9A4252
:1065700009D14FF0500080F31188BFF36F8FBFF344
:106580004F8F00BFFEE7D0F800298A4209D14FF0B3
:10659000500080F31188BFF36F8FBFF34F8F00BFA0
:1065A000FEE7017844F6F4720191FF210170017851
:1065B000C2F200028DF803109DF8031001F05001A3
:1065C000117044F6F871C2F2000107220A609DF9C9
:1065D0000320B2F1FF3F0CDC0A6800BF9DF80330D6
:1065E000013A5B008DF803309DF90330002BF5D4A0
:1065F0000A600A68032A2DD14FF4E06303EA0222FD
:106600000A6001990170D0F8201941F47001C0F8B6
:106610002019D0F8201941F07041C0F82019FFF777
:10662000EDFC40F21410C2F2000000210160FFF7FF
:1066300059FC4EF63470CEF20000016841F0404142
:106640000160FFF72FF9FFF737FFFFF7BBFA0020D4
:1066500002B080BD4FF0500080F31188BFF36F8F00
:10666000BFF34F8FFEE7000080B54FF0500080F37E
:106670001188BFF36F8FBFF34F8F00F043FE30B12F
:106680004EF60450CEF200004FF080510160002021
:1066900080F3118880BD000010B502460120002162
:1066A00000F018F80446FEF7F1FF204610BD000088
:1066B00010B582B00B468446012000210022CDF89F
:1066C00000C000F02BF80446FEF7E0FF204602B0C1
:1066D00010BD0000F0B581B0B0B105464843503060
:1066E00014460E46FFF7CEFA074650B1002007F1D8
:1066F000500287F846002846314623460097FEF7A9
:10670000D5FF384601B0F0BD4FF0500080F311883E
:10671000BFF36F8FBFF34F8FFEE70000B0B582B0BD
:1067200068B11D46ABB1F1B9EAB14FF0500080F34A
:106730001188BFF36F8FBFF34F8F00BFFEE74FF09D
:10674000500080F31188BFF36F8FBFF34F8F00BFEE
:10675000FEE74FF0500080F31188BFF36F8FBFF357
:106760004F8F00BFFEE751B14AB94FF0500080F3A0
:106770001188BFF36F8FBFF34F8F00BFFEE7502329
:106780000193019B502B0AD1069B019C012485F8A3
:1067900046400095FEF78AFF284602B0B0BD4FF094
:1067A000500080F31188BFF36F8FBFF34F8F00BF8E
:1067B000FEE7000070B5F8B104460E46FFF79CFBFB
:1067C0002068D4E90F12002502FB0103013901FB07
:1067D0000201A563C4E90103FF20E16084F84400DD
:1067E00084F8450004F110007EB1FFF73FFB04F18F
:1067F0002400FFF73BFB18E04FF0500080F31188B6
:10680000BFF36F8FBFF34F8FFEE7016869B100F0F0
:10681000FFFE50B14EF60450CEF200004FF0805112
:106820000160BFF34F8FBFF36F8FFFF789FB01202C
:1068300070BD00002DE9F04F83B00292B8B11D4643
:106840000E460446E9B1022D03D1E06B012840F069
:106850009A8000F033FD00BB0298F0B14FF0500079
:1068600080F31188BFF36F8FBFF34F8FFEE74FF0B8
:10687000500080F31188BFF36F8FBFF34F8F00BFBD
:10688000FEE7206C0028DED04FF0500080F3118826
:10689000BFF36F8FBFF34F8FFEE7FFF72DFBA06BAA
:1068A000022D58D0E16B884255D304F11008012025
:1068B0006F464FF0000B0DF108094FF0805A00BFF2
:1068C0000299002900F07B80C00702D03846FFF70C
:1068D000F7FCFFF735FBFFF7E7FDFFF70DFB94F83B
:1068E0004400FF2808BF84F844B094F84500FF280E
:1068F00008BF84F845B0FFF723FB3846494600F04F
:106900000FFB00285ED12046FEF7BEFFA0B1029922
:106910004046FFF7EBFC2046FFF77AF900F0C0FE97
:1069200078B94EF60450CEF20000C0F800A0BFF3D4
:106930004F8FBFF36F8F04E02046FFF769F900F037
:10694000AFFEFFF7D9FAA06B022D04D0E16B8842AD
:106950004FF00000B4D2204631462A46FEF7D0FD63
:1069600054F8241FC9B1204600F052FE08B34EF679
:106970000450CEF200004FF080510160BFF34F8F02
:10698000BFF36F8F15E04FF0500080F31188BFF315
:106990006F8FBFF34F8F00BFFEE750B14EF604502C
:1069A000CEF200004FF080510160BFF34F8FBFF374
:1069B0006F8FFFF7C5FA012003B0BDE8F08FFFF736
:1069C000BFFA04E02046FFF723F900F069FE00203B
:1069D00003B0BDE8F08F00002DE9F04381B0E8B1CD
:1069E0001E46914605460F4609B3022E02D1E86BBA
:1069F000012837D1FFF71CFBEFF311884FF050004F
:106A000080F31188BFF36F8FBFF34F8FA86B022EF7
:106A100019D0E96B884216D300203FE04FF05000B8
:106A200080F31188BFF36F8FBFF34F8FFEE7286CA1
:106A30000028DAD04FF0500080F31188BFF36F8F39
:106A4000BFF34F8FFEE795F84540A86B28463946BF
:106A50003246FEF755FDFF2C0DD0601C85F8450031
:106A600001201BE04FF0500080F31188BFF36F8FBF
:106A7000BFF34F8FFEE755F8240F70B1284600F0A2
:106A8000C7FD0146B9F1000F4FF0010006D0002903
:106A90001CBF0120C9F8000000E0012088F3118824
:106AA00001B0BDE8F0830000B0B5A8B18568044628
:106AB00000F0FEFB85421CBF0020B0BDE06801383D
:106AC000E0601CBF0120B0BD204600210022002351
:106AD000FFF7B0FE0120B0BD4FF0500080F31188E9
:106AE000BFF36F8FBFF34F8FFEE700002DE9F04F2C
:106AF00085B0049298B10C460546002900F0A580A7
:106B000000F0DCFBA8B9049898B14FF0500080F376
:106B10001188BFF36F8FBFF34F8F00BFFEE74FF0B9
:106B2000500080F31188BFF36F8FBFF34F8F00BF0A
:106B3000FEE705F1240005F11009019002AF0DF107
:106B4000100A4FF000080AE02846FFF761F800F04D
:106B5000A7FD2846FEF78CFE002840F08480FFF752
:106B6000CBF9D5F838B0BBF1000F1DD0284621462F
:106B7000FEF7B2FCABF10100A863286970B148468A
:106B800000F046FD50B14EF60450CEF200004FF03A
:106B900080510160BFF34F8FBFF36F8FFFF7D0F9C4
:106BA00000200126A0B95FE0049850B1B8F1000FB1
:106BB00002D13846FFF784FB4FF00108012038B9B5
:106BC00052E0FFF7BDF90026002000284CD000BF9E
:106BD000FFF7B6F9FFF768FCFFF78EF995F8440068
:106BE000FF2804BF002085F8440095F84500FF28E1
:106BF00004BF002085F84500FFF7A2F9384651464A
:106C000000F08EF900289FD12846FEF731FEB0B182
:106C100004990198FFF76AFB2846FEF7F9FF00F098
:106C20003FFD00289BD14EF60450CEF200004FF0FD
:106C300080510160BFF34F8FBFF36F8F8FE72846FE
:106C4000FEF7E6FF00F02CFD89E7286C00283FF4F2
:106C500057AF4FF0500080F31188BFF36F8FBFF331
:106C60004F8F00BFFEE70026304605B0BDE8F08F2D
:106C70002DE9F04381B000B3914605460E4631B38D
:106C8000FFF7D6F9EFF311884FF0500080F3118829
:106C9000BFF36F8FBFF34F8FAC6B24B395F8447085
:106CA00028463146FEF718FC601EFF2FA8631CD053
:106CB000781C85F8440001202AE04FF0500080F352
:106CC0001188BFF36F8FBFF34F8F00BFFEE7286CB3
:106CD0000028D5D04FF0500080F31188BFF36F8F9C
:106CE000BFF34F8FFEE7002012E055F8100F70B190
:106CF000284600F08DFC0146B9F1000F4FF001006D
:106D000006D000291CBF0120C9F8000000E00120C6
:106D100088F3118801B0BDE8F08300002DE9F04F41
:106D200085B0049158B10446006C90B14FF050000A
:106D300080F31188BFF36F8FBFF34F8FFEE74FF0E3
:106D4000500080F31188BFF36F8FBFF34F8F00BFE8
:106D5000FEE700F0B3FA50B9049840B14FF050008C
:106D600080F31188BFF36F8FBFF34F8FFEE704F1FD
:106D7000240004F1100501904FF0000802AF0DF15E
:106D8000100A4FF000094FF0000B0AE02046FEF712
:106D90003FFF00F085FC2046FEF76AFD002840F02A
:106DA0007F80FFF7A9F8A06BF0B10138A0632068DD
:106DB00010B9FFF70DF8A060286870B1284600F000
:106DC00027FC50B14EF60450CEF200004FF0805137
:106DD0000160BFF34F8FBFF36F8FFFF7B1F801264C
:106DE0000020B8B96FE000BF049850B1BBF1000FAC
:106DF00002D13846FFF764FA4FF0010B012048B981
:106E000061E0B9F1000F62D1FFF79AF80020002687
:106E1000002858D0FFF794F8FFF746FBFFF76CF80F
:106E200094F84400FF2808BF84F8448094F8450093
:106E3000FF2808BF84F84580FFF782F8384651469E
:106E400000F06EF80028A1D12046FEF711FD28B908
:106E50002046FEF7DDFE00F023FCA2E7206838B9EB
:106E6000FFF74AF8A06800F089FB8146FFF768F851
:106E700004990198FFF73AFA2046FEF7C9FE00F0A0
:106E80000FFC00287FF48DAF4EF60450CEF20000C8
:106E90004FF080510160BFF34F8FBFF36F8F80E7DA
:106EA000B9F1000F0ED0FFF727F82046FEF782FB5E
:106EB000A168024608461146FFF752FAFFF740F86C
:106EC000002600E00026304605B0BDE8F08F4FF008
:106ED000500080F31188BFF36F8FBFF34F8F00BF57
:106EE000FEE7000070B568B1866804460D4600F004
:106EF000DFF986420FD020462946FFF70FFF58B929
:106F0000002070BD4FF0500080F31188BFF36F8FE9
:106F1000BFF34F8FFEE70120E1680131E16070BDF2
:106F2000B0B5D0B10D4611B30446FEF7E5FF45F20A
:106F3000C870C2F2000001682868421C21D045F2E6
:106F400030736268C2F20003D3F800C091421AD3D2
:106F500023689C4517D0012422E04FF0500080F3B5
:106F60001188BFF36F8FBFF34F8F00BFFEE74FF065
:106F7000500080F31188BFF36F8FBFF34F8F00BFB6
:106F8000FEE700240CE0891A884206D9401A2860DE
:106F90002046FFF795F9002402E000200124286034
:106FA000FEF7CEFF2046B0BD2DE9F04383B0074683
:106FB0009000984615468946FEF764FE78B106466D
:106FC0005C20FEF75FFE38B10446066354B94FF00B
:106FD000FF3003B0BDE8F0833046FEF7C9FF002460
:106FE000002CF4D0DDE90A10002284F85920CDE904
:106FF0000010384649462A4643460294FEF766FB8F
:107000002046FEF7ADF9012003B0BDE8F083000093
:1070100070B586B00B9CCCB10C9E06B35C25049574
:10702000049D5C2D25D1049DDDF828C0022586F83D
:10703000595005AD3463CDE900C50296FEF746FB15
:107040003046FEF78DF9059806B070BD4FF0500040
:1070500080F31188BFF36F8FBFF34F8FFEE74FF0C0
:10706000500080F31188BFF36F8FBFF34F8F00BFC5
:10707000FEE74FF0500080F31188BFF36F8FBFF32E
:107080004F8F00BFFEE70000F0B581B0D0B11D46C4
:10709000174604460E46FEF72FFF002D1CBF606DFD
:1070A000286094F858000221042F84F8581012D850
:1070B0000125DFE807F023031C262000616D314322
:1070C00061651FE04FF0500080F31188BFF36F8FB0
:1070D000BFF34F8FFEE7616D013113D04FF05000C9
:1070E00080F31188BFF36F8FBFF34F8FFEE7616DA1
:1070F0000131616506E0022803D1002501283CD159
:1071000003E066650125012837D1261D3046FEF7CC
:107110007FFE45F21001C2F20001E06A0A68904267
:1071200088BF086040F2405100EB8000C2F20001CD
:1071300001EB80003146FEF7C7FEA06A48B14FF070
:10714000500080F31188BFF36F8FBFF34F8F00BFE4
:10715000FEE740F22851C2F20001E06A0968C96AFC
:1071600088420AD94EF60450CEF200004FF080510A
:107170000160BFF34F8FBFF36F8FFEF7E1FE28462C
:1071800001B0F0BD2DE9F04120B31D46174604467D
:107190000E46FEF74DFFEFF311884FF0500080F3DD
:1071A0001188BFF36F8FBFF34F8F002D1CBF606D31
:1071B000286094F858000221042F84F8581012D83F
:1071C0000125DFE807F023031C262000616D314311
:1071D00061651FE04FF0500080F31188BFF36F8F9F
:1071E000BFF34F8FFEE7616D013113D04FF05000B8
:1071F00080F31188BFF36F8FBFF34F8FFEE7616D90
:107200000131616506E0022803D10025012849D13A
:1072100003E066650125012844D1A06A48B14FF01A
:10722000500080F31188BFF36F8FBFF34F8F00BF03
:10723000FEE745F20800C2F20000006830B145F2F6
:10724000407004F11801C2F2000015E0261D30461E
:10725000FEF7DEFD45F21001C2F20001E06A0A68A5
:10726000904288BF086040F2405100EB8000C2F2BB
:10727000000101EB80003146FEF726FE40F2285166
:10728000C2F20001E06A0968C96A88420AD9069810
:1072900000281CBF0121016045F2D470C2F2000039
:1072A0000121016088F311882846BDE8F0810000C3
:1072B00040F22850C2F200000068704745F2947016
:1072C000C2F200000068002804BF0120704745F2A8
:1072D0000800C2F200000068B0FA80F040094000E7
:1072E0007047000045F2C870C2F2000000687047A5
:1072F00080B5FEF79DFE45F2C870C2F2000000683E
:1073000080BD00002DE9F04F81B045F20800C2F2C7
:107310000000006840B145F23C70C2F20000016814
:1073200000240131016092E045F2C870C2F2000011
:1073300001684E1C066021D340F23050C2F20000BA
:107340000168096849B14FF0500080F31188BFF31C
:107350006F8FBFF34F8F00BFFEE740F23852C2F28B
:10736000000201681368036045F230701160C2F2D8
:107370000000016801310160FEF7B2FB45F22C719B
:10738000C2F20001086840F2285A40F24058864292
:10739000C2F2000AC2F2000801D2002445E040F225
:1073A0003057C2F2000738680024006898B345F2ED
:1073B000100BC2F2000B19E0D9F82C00DBF800101A
:1073C000884288BFCBF8000000EB800008EB80000B
:1073D0002946FEF779FDD9F82C00DAF80010C96AC1
:1073E0003A68884228BF01241068B8B13868C0687C
:1073F000D0F80C904D4655F8040F864210D328461D
:10740000FEF706FDD9F828000028D5D009F11800AC
:10741000FEF7FEFCD0E74FF0FF3005E04FF0FF3005
:1074200045F22C71C2F200010860DAF80000C06A6F
:1074300000EB800058F82000012845F2D470C2F219
:10744000000088BF01240068002818BF01242046DE
:1074500001B0BDE8F08F00002DE9F0411E46154651
:1074600088460746FEF748FD40F22854C2F2000461
:10747000206890F85800022819D02068416D21EA50
:107480000701416520684FF0010180F8581076B17E
:1074900030460121FDF724FF4EF60450CEF20000E5
:1074A0004FF080510160BFF34F8FBFF36F8FFEF736
:1074B00047FDFEF721FD15B12068406D286020686A
:1074C000002590F858100020022905D121680125D7
:1074D0004A6D22EA08024A65216881F85800FEF7E1
:1074E0002FFD2846BDE8F081B0B580B1044640F2DA
:1074F0002850C2F200000068A0420AD04FF05000AD
:1075000080F31188BFF36F8FBFF34F8FFEE700202A
:10751000B0BD206D38B3013820654FF0000018BFB2
:10752000B0BDE16AE26C91421CD0251D2846FEF7F1
:107530006FFCE06CC0F13801A16145F21001E0621E
:10754000C2F200010A68904288BF086040F24051D0
:1075500000EB8000C2F2000101EB80002946FEF73B
:10756000B3FC0120B0BD4FF0500080F31188BFF391
:107570006F8FBFF34F8F00BFFEE70000F0B581B003
:1075800000B340F22856C2F200060446C06A3168D1
:10759000C96A884219D2A169002904D43168C96A2C
:1075A000C1F13801A16140F24057616900EB8000F0
:1075B000C2F2000707EB800081420FD03068C06A3A
:1075C000E06221E0002001B0F0BDE16C3068C26AE9
:1075D0000020914238BF012001B0F0BD251D284692
:1075E000FEF716FC306845F21001C06AC2F20001D5
:1075F000E0620A68904288BF086000EB800007EBF9
:1076000080002946FEF760FC012001B0F0BD0000BB
:10761000B0B5C068C5687DB105F118042046FEF715
:10762000F7FB45F20800C2F20000006868B145F2BD
:107630004070C2F200001DE04FF0500080F311884E
:10764000BFF36F8FBFF34F8FFEE72C1D2046FEF771
:10765000DFFB45F21001C2F20001E86A0A689042BD
:1076600088BF086040F2405100EB8000C2F2000188
:1076700001EB80002146FEF727FC40F22851C2F2C0
:107680000001E86A0968C96A884291BF002045F292
:10769000D471C2F20001012088BF0860B0BD0000B3
:1076A0002DE9F04F81B045F20804C2F200042068D1
:1076B00068B1FEF721FC206801382060206880B1A5
:1076C0000024FEF73DFC204601B0BDE8F08F4FF0EE
:1076D000500080F31188BFF36F8FBFF34F8F00BF4F
:1076E000FEE745F20000C2F20000006800285DD00D
:1076F00045F24076C2F20006306845F2D478C2F214
:10770000000890B345F2100740F2405940F2285B60
:10771000C2F20007C2F20009C2F2000B4FF0010AE8
:10772000F068C56805F11800FEF772FB2C1D2046B5
:10773000FEF76EFBE86A3968884288BF386000EB64
:10774000800009EB80002146FEF7BEFBE86ADBF80B
:107750000010C96A884228BFC8F800A03068002815
:10776000DED1002D18BFFEF7BBF945F23C74C2F222
:107770000004256855B10126FFF7C4FD002818BF95
:10778000C8F80060013DF7D100202060D8F8000063
:1077900070B14EF60450CEF200004FF080510160FF
:1077A000BFF34F8F0124BFF36F8F8AE7002488E770
:1077B000002486E780B586B0FDF728FE45F2CC7040
:1077C000C2F20000006808B30020CDE9040005A85B
:1077D00004A903AAFEF73CFBDDE903200221DDF842
:1077E00014C0CDE9001045F6F930C0F600000CA138
:1077F0000023CDF808C0FFF70BFC45F2D071C2F2B0
:107800000001086010B1012006B080BD4FF05000AB
:1078100080F31188BFF36F8FBFF34F8FFEE700BF78
:10782000546D72205376630010B584B0A8B145F250
:10783000CC74C2F2000484462068C0B10529CDE9A9
:107840000012CDF808C015DCFFF738FD01462068AE
:10785000022916D1069A694615E04FF0500080F3D0
:107860001188BFF36F8FBFF34F8F00BFFEE700207B
:1078700004B010BD69461A460023FFF7ADF804B006
:1078800010BD694600220023FEF7D4FF04B010BDEE
:107890004100080218BF04200A0E18BF40F0010082
:1078A0004FF07F4232EA010108BF40F00200012898
:1078B00008BF05207047000000B510EE101A2DED2E
:1078C000028B81B04D4A6846B2EB410F3CD94FF074
:1078D000E640B0EB410F94BF00204FF0FF30009026
:1078E0000098B0EE408A00285FDB28EE080ADFED42
:1078F000440A9FED441A00EE201ADFED430A40EEE1
:10790000010A9FED421A00EE201ADFED410A10F045
:10791000010F40EE010A9FED3F1A00EE201A61EEC2
:10792000000AB0EE480A08EE200A02BF01B0BDEC22
:10793000028B00BDBFEE001A01B0C1EE000ABDEC23
:10794000028BB0EE600A00BD334B21F0004293423F
:1079500028D911F0004FDFED310A20EE201ADFEDBB
:10796000300A19BF31EE601A71EE200A31EE201A8A
:1079700071EE600ABDEEE01A11EE100A9FED291AB1
:1079800000F0030000EEC10A9FED271A009000EE00
:10799000C10A9FED261A00EEC10A9FED251A00EEDE
:1079A000C10A9DE700F05AF89AE718EE100A400065
:1079B000B0F17F4F0DD218EE100AFFF769FF0428CF
:1079C00008BF00F043F8B0EE480A01B0BDEC028BEE
:1079D00000BD09D10120F8F76DFD01B0BDEC028BAF
:1079E0005DF804EB00F02AB801B0B0EE480ABDEC37
:1079F000028B5DF804EB00F01DB80000B61F927E0C
:107A0000BCE9223C0B6D063B8A76CE3CACB5593DB9
:107A100035A1083E29AAAA3E490E494683F9223FCC
:107A20000000004B0000C93F00A0FD390020A23338
:107A30001A61342C30EE000A70470000DFED020AB4
:107A400080EEA00A70470000000000009FED020ACF
:107A500020EE000A70470000000000102DE9F00140
:107A60004FF07F42B2EB410F9FBF4FF0FF310160FB
:107A7000BDE8F00170474FF0004242EA0123C1F334
:107A8000C752783A551112F01F0C434CCCF1200626
:107A90007C44C1F3C752A2F178024FEA621204EBB0
:107AA000820254F8254008BFD2E9015612D0556829
:107AB00004FA0CF425FA06F73C43976805FA0CF52E
:107AC00027FA06F8D26807FA0CFCF24045EA0805E6
:107AD0004CEA0206A4FB034CA5FB0352A6FB03637E
:107AE0001D449D4234BF012600261319334416B1AC
:107AF000934202D903E0934201D2012200E0002226
:107B0000624402F1200C9206DC0C42EA443200EEA0
:107B1000102A5B03DFED210AF8EEC01A00EE103ADE
:107B20004FEA9C1C11F0004FB8EE400AC0F800C0AC
:107B300020EE201A00EE105ADFED190AB8EE400AC6
:107B400020EE200A71EE810A70EE800A10EE902A73
:107B500002F500626FF30B0200EE902A70EEE11A5C
:107B600031EEC11ADFED101A30EE411A9FED0D0A09
:107B700020EE800A01EE210A9FED0C1A00EE810A28
:107B800004BFBDE8F0017047CCF180510160BDE851
:107B9000F001B1EE400A70477405000000000036A5
:107BA0000000802C22AAFD29DB0FC92F0000C92F5D
:107BB0002DE9C04130B4DFF8A4C23CEA111418BF6B
:107BC0003CEA131400F0ED801CEA111481EA03056D
:107BD00044EAD57418BF1CEA131500F0C880A4EB62
:107BE000050404F17F7404F500344FF0004545EAC4
:107BF000C12145EAC32341EA505143EA52534FEAB7
:107C0000C0204FEAC222994208BF904200F09D80F6
:107C10004FEA13650FF24416765D4FEA134506FBF3
:107C200005F7C7F1807706FB07F74FEAD737A7FBC1
:107C300003687642A7FB06CEC8F5803838BFA8F1A6
:107C4000010807FB08E6A6FB028C4FF0000EE6FBDE
:107C500003CEDCF1000CCEF1004E38BFAEF1010EC8
:107C6000A6FB0C584FF00007E6FB0E87A1FB08C6E9
:107C7000A0FB07CE16EB0E064FF0000545F1000500
:107C8000E1FB076515F1E04E7EBFA4F580345FEAA5
:107C900046066D4116F1800745F100054FEA1727AA
:107CA00047EA05674FEA15254FEA0666A6F1DE4664
:107CB000B6F1805F20D9384605EBC47124F0010C81
:107CC00001EB0C11BCF1FE6F02D8F0BCBDE80081E5
:107CD00024425CBF01F5801E9EEAC47F02D4F0BC42
:107CE000BDE80081244200F13980A1F1C041F0BC1F
:107CF000BDE8004100F044B94FEAD02040EA4150CD
:107D00004FEAD1214FEAD22242EA43524FEAD3232B
:107D1000A7FB028607FB036605FB02661EEA0E0F41
:107D200058BFA6EB0056B6EB00564FEA520E4EEA8D
:107D3000C37E18EB0E0E56EB530EBCD518EB0208A3
:107D40005E417F1C55F10005B5E74FF480154FF0FB
:107D500000074FF000064FF00008ACE701F1C0410A
:107D600001F000414FF00000F0BCBDE800810CEADA
:107D7000131511EA0C1F00D00CE013EA0C1F00F0E1
:107D800026804FF0000081EA030101F00041F0BCC1
:107D9000BDE80081F0BCBDE8004181EA030100F0CC
:107DA000EFB8F0BCBDE8004170B500F09BF800BF33
:107DB000097EFC3E00F007B84FF0000081EA0301A5
:107DC00001F00041704781EA030100F0D9B8F0BC2E
:107DD000BDE8004122494FF000007047FFFDFBF96C
:107DE000F7F5F4F2F0EEEDEBE9E8E6E4E3E1E0DEEE
:107DF000DDDBDAD8D7D5D4D3D1D0CFCDCCCBCAC860
:107E0000C7C6C5C4C2C1C0BFBEBDBCBBBAB9B8B786
:107E1000B6B5B4B3B2B1B0AFAEADACABAAA9A8A879
:107E2000A7A6A5A4A3A3A2A1A09F9F9E9D9C9C9B47
:107E30009A999998979796959594939392919190F2
:107E40008F8F8E8E8D8C8C8B8B8A89898888878783
:107E50008685858484838382828181800000FF07F8
:107E60000000F87F4FEA1153A3F58063D3F11E039E
:107E7000A8BFD3F1200C08DB4FF0004242EAC12238
:107E800052EA505232FA03F0704709420BD4102BD9
:107E9000C4BF0020704703F5787CBCF1FF3F05D0DC
:107EA0004FF0FF3070474FF00000704770B500F0A2
:107EB00019F800BF4992248000207047F0E7B0FA1B
:107EC00080F310FA03F10AD0C3F11D0303F58063B8
:107ED0004FEA03524FEA415002EBD12170474FF075
:107EE000000070470EF1020E2EF0030E5EF8046BD8
:107EF000364205D4012A43EB030515F5001F12D8BD
:107F0000012841EB010C1CF5001F0CD80ED14FEAE3
:107F1000D17C0CEB4C0C0CF1020C15F5001F08BFCA
:107F20004CEBD37C04E04FF0080C01E04FEAD37C2B
:107F30000CEB4C0526FA05F606F00706B6F1040C24
:107F400006D20EEB860CBDE870404CF0010C604789
:107F5000DFE80CF0090B02024FF00041A1F500210F
:107F60004FF0000070BD19461046012851EB010486
:107F700018BFD4F5001484BF002001F0004170BD8B
:107F80000808A0F500114FEA310170474FF07E520A
:107F900009E011F0004204D54042C1F1000138BFB0
:107FA000491E42F07E5202F170620B0012BF202384
:107FB0005FEA00017047B1FA81FC01FA0CF1A3EB12
:107FC0000C0320FA03FC41EA0C0102EBC352C3F19B
:107FD000200310FA03FC5CEA416C42EB112018BF4D
:107FE0005FF0806C28BF20F001007047F1EE100AAE
:107FF0004FF6FF71C0F2C03120EA010040F040703E
:10800000E1EE100A70470000000000006E83F9A244
:108010002915444ED15727FCC0DD34F5999562DB14
:108020004190433CAB6351FE0000000000000000A3
:10803000010203040607080900000000010203040E
:10804000EA800008000000000000000000000000BE
:1080500000000000000400003000000000000000EC
:1080600000000000DC8000080000000000000000AC
:1080700000000000000000000004000018000000E4
:108080000000000000000000DF8000080000000089
:1080900000000000000000000000000000080000D8
:1080A000180000000000000000000000D080000860
:1080B00000000000000000000000000000000000C0
:1080C0000002000018000000000000000000000096
:1080D00064656661756C745461736B0072630073E0
:1080E000686F6F745F6374726C005461736B5F4987
:1080F0006E6974001881000800000020180100005B
:10810000C40100083082000818010020C05C000093
:10811000E0010008000000000024F400010000005D
:10812000060000000000803F050000000000803FC6
:10813000030000000100000000000000010000003A
:10814000000070430000003F000000000000070234
:10815000010001000000803F6666E63FCDCCCC3DCB
:10816000CDCC4C3DCDCCCC3D6666663F0000F041A9
:10817000000080BF0000803F00008040CDCCCC3E9E
:108180000AD7233D0000803E0AD7233C000020424E
:10819000000080BF000020400000803FCDCCCC3DDF
:1081A0000AD7233DCDCCCC3E0000803F000080BFED
:1081B000DB0FC9400000803F0000C03F9A99993E04
:1081C0000000003FCDCC4C3E0000803F000080BF4F
:1081D000000080BF0000003F6666E63F9A99993E26
:1081E000CDCCCC3D9A99193E0000803F000080BF65
:1081F000DB0FC9400000803F0000803F000000000E
:1082000000000000000000000000803F000080BF70
:10821000000080BF0000F0410000F0410000F0418C
:108220000000F0410100000010000000AAAAAAAA64
:040000050800018965
:00000001FF
